:1000000000400020DD4400001D4500001F450000A9
:1000100000000000000000000000000000000000E0
:10002000000000000000000000000000214500006A
:1000300000000000000000002345000025450000EE
:100040002745000027450000114D0000274500000E
:10005000274500000000000027450000274500005C
:1000600027450000554700002745000027450000B0
:1000700027450000274500002745000027450000D0
:1000800027450000B54D000027450000274500002A
:1000900027450000274500002745000027450000B0
:1000A0002745000027450000000000000000000078
:1000B0000000000000000000000000000000000040
:1000C000054B0648033310B51B1A062B03D9044B06
:1000D000002B00D0984710BD14020020140200200D
:1000E000000000000648074910B5091A8910CB0F17
:1000F0005918491003D0044B002B00D0984710BD6D
:1001000014020020140200200000000010B5074C6B
:100110002378002B09D1FFF7D3FF054B002B02D02A
:10012000044800E000BF0123237010BD140200202A
:1001300000000000B4740000094B10B5002B03D080
:100140000849094800E000BF08480368002B02D1B5
:10015000FFF7C8FF10BD064B002BF9D09847F7E713
:100160000000000018020020B474000010020020FB
:1001700000000000164B002B00D1144B9D4640227E
:1001800092029A1A924600218B460F461348144A4F
:10019000121A05F07EF80F4B002B00D098470E4B3B
:1001A000002B00D098470020002104000D000D48CE
:1001B000002802D00C4800E000BF05F027F820001E
:1001C000290004F0BDFD04F0FBFFC046000008005C
:1001D0000040002000000000000000001402002089
:1001E0003424002000000000000000000123034030
:1001F0000200181E04D1042A03D91068000900E087
:100200000020704710B50400FFF7F0FF0300002046
:1002100083420BD0013B9B00181DE2181279002A83
:1002200003D001338342F8D100E0180010BD012251
:10023000016810B5114201D0002903DA102000F046
:10024000E3F903E04910062001F004FF10BD016846
:1002500010B5CB0701D5002903DA102000F0D4F93E
:1002600006E04910033189100022052001F0F2FE5A
:1002700010BD70B50568AB0728D1042D26D90F2312
:100280002A6846681340062B09D12800FFF7AEFF05
:10029000012383421DDC9A00AE500133F9E7052BA0
:1002A00014D1F30703D4132000F0AEF912E0761056
:1002B000FF2EF8D82800FFF799FF2C1D230080009F
:1002C0002018984205D91E700133FAE70B2000F080
:1002D0009BF9002070BD70B50468E30701D41120BC
:1002E0002DE04568AB0729D1042D27D90F262B68AF
:1002F00064101E40062E0BD1002C04DD2800FFF7F1
:1003000075FF844201DD122019E0A400605918E055
:10031000331F012B12D82800FFF768FF8000042E3E
:1003200002D12800FFF76EFF002CECDDA042EADBD3
:1003300001232C19E0784000184302E00B2000F064
:1003400063F970BDF8B5012304681C4201D1112086
:100350002FE00325466835402AD1042E28D90F23E3
:100360003268641087681340062B0BD1002C04DD23
:100370003000FFF73BFF844201DD122019E0A400AA
:10038000A75113E0052B13D1002CF6DD3000FFF749
:100390002DFF80008442F0DC01231F4201D1132095
:1003A00007E07F10FF2FFAD83419E770280002E029
:1003B0000B2000F029F9F8BD006810B5830717D1AC
:1003C000042815D90F2302681340062B02D1FFF72A
:1003D0000DFF0BE0052B05D1FFF708FFC00001233F
:1003E000184308E0042B03D1FFF70CFF4000F6E7A9
:1003F0000B2000F009F910BD10B50324006804407B
:1004000006D1042804D90F2302681340042B01D01D
:100410000E2011E001F05AFE0378233B5942594166
:1004200010224018210005F00DFC80239B05C21806
:10043000054B9A4203D9142000F0E6F802E00123AC
:100440004000184310BDC046FFFFFF3F10B5012418
:100450000368234202D04268224203D10D2000F0FB
:10046000D3F808E004495B1052101B070A401343FD
:1004700018684000204310BDFCFFFF0F01210368F6
:1004800010B50B4205D042680A4202D0806808428B
:1004900003D10D2000F0B8F808E005495B105210B8
:1004A0001B070A40401013431860002010BDC046CF
:1004B000FCFFFF0F012303400200181E01D0501063
:1004C00002E00D22014B1A707047C0463002002036
:1004D000012303400200181E04D1042A03D9106826
:1004E000000900E00020704770B50D000400FFF720
:1004F000EFFF86002800FFF7EBFF830000209E42FD
:100500000ED1231D9E1904351A009E4207D9297861
:100510001278013301358A42F6D0002000E0012034
:1005200070BD0000F0B585B00393019002912D4E8F
:100530002D4B002A02D002223270013A00251A60A7
:100540001B68F554019B9D424ADA029AAB00D058D1
:10055000254B1C68C8239B0037191C1B012318421C
:1005600002D04310214A1FE0214A002802D004286B
:1005700005D1204A2100380005F052FA18E004287D
:1005800010D90F2302681340042B04D101F09EFD03
:10059000194A030008E0062B05D1FFF799FF174A17
:1005A000030001E00123164A2100380005F038FA63
:1005B000300005F09BFA039B0B4A002B01D1106021
:1005C0000CE0019B013B9D42F9DA0E4B9842F6DCB0
:1005D000431C1360202232540022F2540135B1E74B
:1005E00005B0F0BD3C02002038020020116A000076
:1005F000E4690000EA690000186D0000EF6900007E
:10060000006A00001F030000014B187000207047B3
:100610003002002070B502F07BFE094C0100251D60
:100620001F22280005F069FA280005F05FFA04236C
:1006300004308008000118432060200070BDC046CF
:100640005C050020C368F0B59D00836887B05D1924
:10065000030018330393036902909F00039BDF1983
:1006600043699E000093039B9E19D24B1B78002B7D
:100670000FD17F222B68D0491C1213409B005B587E
:1006800000960435019235E0CA4B1B78002B29D027
:10069000009E029BC74C9B6821780093EA1A029B3C
:1006A00092109B7812021A43029B587802F0BCFB0E
:1006B0000023029A2370137000960497029B039AFA
:1006C0009B68ED1A0193029BAD10DD60049B9F1A9D
:1006D000029BBF101F61009B9B1A029A9B105361E3
:1006E00001F005FC2B68019A1C121340B24A9B00D2
:1006F0009B5804359F46029B587802F08DFB0023DF
:10070000029A1370D9E7039B3A1DD11AA94BDB2932
:1007100003DD1A22009E1A70BBE71B783C60002B99
:1007200002D0009E1700B4E72B6801991C120B4001
:10073000A1499B005B5817000435DBE7039B3A1D7A
:10074000D11A9C4BDB2903DD1A22009E1A70A0E708
:1007500028681B78291D3860002B03D0009E1700E5
:100760000D0096E76B6801991C120B4092499B00A3
:100770005B5817000835BDE7039B3A1DD11A8D4B16
:10078000DB2903DD1A22009E1A7082E7A4001B7881
:100790002C193C60002B02D0009E170079E72B68D3
:1007A00001991C120B4084499B005B5817000435CB
:1007B000A0E7039B3A1DD11A7E4BDB2903DD1A22E9
:1007C000009E1A7065E77D48A40021581B783960A7
:1007D000002B02D0009E17005BE72B6801991C12CA
:1007E0000B4075499B005B581700043582E7043FB6
:1007F000724B3A68A400E2506E4B1B78002B01D07C
:10080000009E46E72B68019A1C1213406A4A9B001F
:100810009B5804356EE7694BA600F058FFF74AFE77
:10082000043F04003868FFF745FE24180120634B9D
:1008300064000443F4505F4B1B78002B01D0009EF2
:1008400027E72B68019A1C1213405B4A9B009B58B8
:1008500004354FE7039B3A1DD11A564BDB2903DDC4
:100860001A22009E1A7014E70098039C0121A042EE
:1008700002D901000C3909681B783960002B02D0BD
:10088000009E170005E72B6801991C120B404A498E
:100890009B005B58170004352CE7039B3A1DD11AC7
:1008A000444BDB2903DD1A22009E1A70F1E6009901
:1008B000039881420AD90B000C3B1B6840495B102E
:1008C0006418E41A009BA400E35802E01821197090
:1008D00000233B60374B1B78002B02D0009E170093
:1008E000D7E62B6801991C120B4033499B005B58DB
:1008F00017000435FEE6009B039A93420BD90C3B8C
:1009000019682F4B043FE3184910591A3A68009BA5
:100910008900CA5002E01822264B1A70254B1B781A
:10092000002B01D0009EB4E62B68019A1C121340E4
:10093000214A9B009B580435DCE6009B039A9342B6
:100940001CD9009E1E4B0C3EE4183368009A5B10C5
:10095000E31A9B009858FFF7ADFD043F04903868F8
:10096000FFF7A8FD3168049B4910611A012418188B
:100970004000009B89002043C85002E018220D4B24
:100980001A700C4B1B78002B01D0009E81E62B685F
:10099000019A1C121340084A9B009B580435A9E693
:1009A000039B3A1DD11A034BDB290BDD1A22009E53
:1009B0001A706EE630020020E46700009C220020DE
:1009C000FDFFFF3F0099A40061581B783960002BA0
:1009D00002D0009E17005CE62B6801991C120B40A8
:1009E000CF499B005B581700043583E6043F009B0A
:1009F0003A68A400E250CB4B1B78002B01D0009E3C
:100A000047E62B68019A1C121340C54A9B009B586D
:100A100004356FE6009BA4001C192368043F386866
:100A20005E10FFF747FD36180120BE4B76001B789D
:100A300006432660002B01D0009E2AE62B68019A0F
:100A40001C121340B64A9B009B58043552E6039B88
:100A5000A4003F1BB34CBB420DD82378002B01D020
:100A6000009E16E62B68019A1C121340AC4A9B00AC
:100A70009B5804353EE6AC4801F09EFA2378002BE3
:100A800001D0009E05E62B68019A1C121340A44A6F
:100A90009B009B5804352DE6A300ED18002C00DACE
:100AA0000BE6A04B1B78002B01D0009EF1E52B68D4
:100AB000019A1C1213409A4A9B009B58043519E670
:100AC0003B1F04931B680593042B04D1A300ED186E
:100AD000002C00DAF2E5934B1B78002B02D0009E2D
:100AE000049FD6E52B68019A1C1213408C4A9B0088
:100AF0009B58049F0435FDE53B1F04931B68059339
:100B0000002B04D1A300ED18002C00DAD6E5854BAC
:100B10001B78002B02D0009E049FBAE52B68019A37
:100B20001C1213407E4A9B009B58049F0435E1E54C
:100B30003A1F13685B10013B002B07DD01215B00AE
:100B4000A4000B4304972D191360B7E5754B1700EC
:100B50001B78002B01D0009E9BE52B68019A1C128C
:100B600013406F4A9B009B580435C3E53A00039B32
:100B70000C32D31ADB2B04DD1A226A4B009E1A704A
:100B800087E5FF2361005B000B4001210B433B60C5
:100B9000029B03989B6824120493ED1A029BAD10EC
:100BA0009B782D021D43009B8D401B1A9B108B4090
:100BB0000B43BB60029B0D437D609C70E4B25B4BBA
:100BC000E4000299E35816008B6056490978002921
:100BD00003D008331D0017005BE51D0001999B68D9
:100BE0000C351C120B404E499B005B5800921700BD
:100BF00080E53B1F1E68039A009B93422AD104970D
:100C00000A20F30716D4B3070DD1042E0BD90F23F6
:100C100032681340042B06D1300001F057FA04F07B
:100C200065FF063006E00720042E03D0002E01D019
:100C300080208000643001F09FFE002801D1043D37
:100C40003CE5029B3100587802F000F90023029A3B
:100C5000137033E5009B009A0C3B1B6802995B10F4
:100C60009B005B421F00D3180C3B1E601300083B27
:100C70001B68083FD7195A108A70D2B22B49D2008C
:100C80005B0055589B0A029A9B009560ED18009BEB
:100C9000043B1E68039B7610B6009E19214B1B78FF
:100CA000002B00D0F5E42B68019A1C1213401C4A5B
:100CB0009B009B58009604351CE53B1F1868FFF706
:100CC000F9FBA40006003F1B1E2833DC00280EDCC5
:100CD000144B1B78002B01D0009EDAE42B68019A9C
:100CE0001C1213400E4A9B009B58043502E502F08B
:100CF000F5FA033E361802F0F1FA0D4B801B9842CC
:100D0000F9D8084B1B78002B01D0009EC1E42B685A
:100D1000019A1C121340024A9B009B580435E9E4D7
:100D2000E467000030020020146A0000A41A0020CA
:100D30009F8601000123029A137002F0CFFA029BF2
:100D40000A3886195E60B8E43B1F1868FFF7B2FBEB
:100D5000A40004903F1B00280EDCCF4B1B78002B17
:100D600001D0009E95E42B68019A1C121340CB4AD7
:100D70009B009B580435BDE4C94B049A009E9A42DF
:100D800003DD1D22C44B1A7083E40123029A137001
:100D900002F0A4FAFA23049A9B005343029A0A3BF6
:100DA0001B18536089E4A300FF1A002320001A00D7
:100DB0003900FFF7B7FBBB4EBB4C3168200001F098
:100DC00091FF3168200002F048F8B34B1B78002BEC
:100DD00001D0009E5DE42B68019A1C121340AF4ABB
:100DE0009B009B58043585E4AB4BA4001B783F1B4C
:100DF000002B01D0009E4CE42B68019A1C1213407A
:100E0000A64A9B009B58043574E401F0FBFD01F0F9
:100E10006EF83B1F1868002823D1083B1868C307E9
:100E200001D5401016E083070FD104280DD90F23F8
:100E300002681340062B02D1FFF74AFB0AE0052B9C
:100E400003D1FFF745FB800004E01922924B009E7E
:100E50001A701EE43A0001214300083A0B43136064
:100E600001E040100138002832DD01224300134325
:100E7000391F0B603B00083B1B681341181A3B00ED
:100E80000C3B1B68134203D08018A400904015E06F
:100E9000990717D1042B15D90F211E683140062957
:100EA00006D101308000C358009AA400A35010E07E
:100EB000052907D118180079A4004000009B1043B1
:100EC000E05006E01922744B009E1A70FFF7E1FB18
:100ED0000435714B1B78002B02D0009EFFF7D9FB25
:100EE0002B68019A1C1213406C4A9B009B580435D6
:100EF000FFF700FCA300039AFB189B1ADB2B01DC15
:100F0000002205E01A22644B009E1A70FFF7C1FB15
:100F1000631E002C03DD3A601C000437F8E75E4BCB
:100F20001B78002B02D0009EFFF7B3FB2B68019AC1
:100F30001C121340594A9B009B580435FFF7DAFBFB
:100F4000A3009C46F81A002C04DC1C22524B0026FD
:100F50001A7015E0002103685B1001268A00825890
:100F6000164003D10D224C4B1A7009E052109342E7
:100F700000DD130001318C42EFDC01265B001E43D3
:100F80006346FF1A444B06601B780437002B02D0DF
:100F9000009EFFF77EFB2B68019A1C1213403F4A0C
:100FA0009B009B580435FFF7A5FBA3009C46F81A4D
:100FB000002C04DC1C22384B00261A7015E000219E
:100FC00003685B1001268A008258164003D10D2267
:100FD000314B1A7009E05210934200DA13000131CC
:100FE0008C42EFDC01265B001E436346FF1A2A4B4E
:100FF00006601B780437002B02D0009EFFF749FBE8
:101000002B68019A1C121340244A9B009B580435FC
:10101000FFF770FB3B00083B1868FFF74BFA3B1FDC
:1010200004901868FFF746FA049AA600BC1B002338
:10103000824200DA04332360174BBF1B1B7804374E
:10104000002B02D0009EFFF724FB2B68019A1C1294
:101050001340124A9B009B580435FFF74BFBA3003B
:10106000FE1A04933B00083B1868FFF723FA3B1F66
:1010700004001868FFF71EFAE20FC317A04253419D
:101080009B003360049BFF1A034B04371B78002B33
:101090000CD0009EFFF7FDFA30020020E46700004C
:1010A00080EE3600380200203C0200202B68019AB6
:1010B0001C121340D84A9B009B580435FFF71AFBBB
:1010C0003B00083B18683B1F1968A300884202D107
:1010D000FB1A042222E004281ED90122104201D06A
:1010E000114219D10326304215D10F2302681A404C
:1010F000042A10D131420ED104290CD90A681340B8
:10110000042B08D1FFF7F0F9431E9841A600BE1B3F
:101110008000306003E0A3000022FB1A1A60BF4B7E
:10112000A4001B783F1B0437002B02D0009EFFF762
:10113000B0FA2B68019A1C121340B74A9B009B58C7
:101140000435FFF7D7FA3B00083B18683B1F1968C6
:10115000A300884202D1FB1A002223E004281FD9F1
:101160000122104201D011421AD10326304216D179
:101170000F2302681A40042A11D131420FD10429E9
:101180000DD90A681340042B09D1FFF7ADF903000C
:1011900058425841A600BE1B8000306003E0A30007
:1011A0000422FB1A1A609D4BA4001B783F1B0437D6
:1011B000002B02D0009EFFF76CFA2B68019A1C12DC
:1011C0001340954A9B009B580435FFF793FAA30000
:1011D000FE1A04933B00083B1868FFF76BF93B1FAE
:1011E00004001868FFF766F9E217C30F8442534101
:1011F0009B003360049BFF1A884B04371B78002B3D
:1012000002D0009EFFF745FA2B68019A1C1213408A
:10121000814A9B009B580435FFF76CFA3B00083B62
:101220001868FFF747F93B1F04901868FFF742F969
:10123000049AA600BC1B0023824200DD0433236015
:10124000764BBF1B1B780437002B02D0009EFFF7A4
:1012500020FA2B68019A1C1213406F4A9B009B587E
:101260000435FFF747FA3B1F1B686C4AA400042BA8
:1012700002D13B1B002103E0002B03D104213B1BC7
:10128000196001E00C23137013783F1B0437002B07
:1012900002D0009EFFF7FDF92B68019A1C12134043
:1012A0005D4A9B009B580435FFF724FAA300FC1A03
:1012B00004933B00083B1868FFF7FCF83B1F06004F
:1012C0001868FFF7F7F836180120049B7600FF1A1C
:1012D000524B06431B7826600437002B02D0009E39
:1012E000FFF7D7F92B68019A1C1213404A4A9B005A
:1012F0009B580435FFF7FEF9A300FE1A04933B0048
:10130000083B1868FFF7D6F83B1F04001868FFF782
:10131000D1F8241A0120049B6400FF1A3F4B0443B8
:101320001B7834600437002B02D0009EFFF7B1F920
:101330002B68019A1C121340374A9B009B580435B6
:10134000FFF7D8F9A300FC1A04933B00083B186888
:10135000FFF7B0F83B1F06001868FFF7ABF84643ED
:101360000120049B7600FF1A2C4B06431B78266055
:101370000437002B02D0009EFFF78BF92B68019AEF
:101380001C121340244A9B009B580435FFF7B2F906
:101390003B00083B1868FFF78DF83B1F0490186866
:1013A000FFF788F80100049803F0D2FD0123A400A0
:1013B0003E1B370040001843184B30601B78043741
:1013C000002B02D0009EFFF764F92B68019A1C12D3
:1013D0001340114A9B009B580435FFF78BF93B00E3
:1013E000083B1868FFF766F83B1F04901868FFF782
:1013F00061F80100049803F091FE0123A4003E1B54
:10140000370049001943054B31601B780437002B26
:1014100006D0009EFFF73DF9E4670000300200208F
:101420002B68019A1C121340E74A9B009B58043515
:10143000FFF760F93B1F1868FFF73CF8C317C018A7
:101440005840012340001843E04BA4001B783E1B8A
:101450003060371D002B02D0009EFFF71AF92B6871
:10146000019A1C121340D84A9B009B580435FFF781
:1014700041F9A300FE1A05933068012C03D1FFF750
:1014800019F8049008E0FFF715F804007068FFF7FA
:1014900011F80130031B0493049B002B01DC012392
:1014A000049304F06FFA049903F038FE0C1901213B
:1014B000059B6400FF1AC54B0C431B78346004374E
:1014C000002B02D0009EFFF7E4F82B68019A1C1253
:1014D0001340BD4A9B009B580435FFF70BF9A4004D
:1014E0003E1B3000FEF788FFB84B30601B78371D7D
:1014F000002B02D0009EFFF7CCF82B68019A1C123B
:101500001340B14A9B009B580435FFF7F3F8A30042
:10151000FE1A04933B00083B1868FEF7CBFF3B1F05
:1015200004001868FEF7C6FF04400120049B640015
:10153000FF1AA64B04431B7834600437002B02D0FB
:10154000009EFFF7A6F82B68019A1C1213409E4AD2
:101550009B009B580435FFF7CDF8A300FC1A0493B9
:101560003B00083B1868FEF7A5FF3B1F0600186804
:10157000FEF7A0FF06430120049B7600FF1A934B61
:1015800006431B7826600437002B02D0009EFFF72D
:1015900080F82B68019A1C1213408B4A9B009B58C1
:1015A0000435FFF7A7F8A300FC1A04933B00083B9F
:1015B0001868FEF77FFF3B1F06001868FEF77AFFEA
:1015C00046400120049B7600FF1A804B06431B789F
:1015D00026600437002B02D0009EFFF75AF82B68D4
:1015E000019A1C121340784A9B009B580435FFF760
:1015F00081F83B1F1868FEF75DFFC04301234000E0
:101600001843724BA4001B783E1B3060371D002B23
:1016100002D0009EFFF73DF82B68019A1C12134080
:10162000694A9B009B580435FFF764F8A300FE1A33
:1016300004933B00083B1868FEF73CFF3B1F040087
:101640001868FEF737FF8440012364001C43049BA5
:101650003460FF1A5D4B04371B78002B02D0009ECC
:10166000FFF717F82B68019A1C121340564A9B008B
:101670009B580435FFF73EF8A300FE1A04933B0085
:10168000083B1868FEF716FF3B1F04001868FEF7BA
:1016900011FF0441012364001C43049B3460FF1AC2
:1016A0004A4B04371B78002B02D0009EFEF7F1FF57
:1016B0002B68019A1C121340434A9B009B58043527
:1016C000FFF718F8A4003E1B3000FEF7B0FD3F4BBB
:1016D00030601B78371D002B02D0009EFEF7D9FF2B
:1016E0002B68019A1C121340374A9B009B58043503
:1016F000FFF700F8A4003E1B3000FEF7A8FD334BB7
:1017000030601B78371D002B02D0009EFEF7C1FF12
:101710002B68019A1C1213402B4A9B009B580435DE
:10172000FEF7E8FFA4003F1B3800FEF7A2FD274BA1
:101730001B78002B02D0009EFEF7ABFF2B68019AAE
:101740001C121340204A9B009B580435FEF7D2FF21
:10175000A4003E1B3000FEF7BEFD1C4B30601B7822
:10176000371D002B02D0009EFEF793FF2B68019AD5
:101770001C121340144A9B009B580435FEF7BAFF15
:10178000A4003F1B3800FEF7DDFD104B1B78002B3B
:1017900002D0009EFEF77DFF2B68019A1C121340B9
:1017A000094A9B009B580435FEF7A4FFA4003E1B8A
:1017B0003000FEF701FE054B30601B78371D002B13
:1017C00006D0009EFEF765FFE467000030020020AF
:1017D0002B68019A1C121340E64A9B009B58043563
:1017E000FEF788FF039A3B1D0493E34C9B1ADB2B07
:1017F00004DD1A23009E2370FEF74BFF01F078FDF5
:1018000001234000184323783860002B03D0009E4A
:10181000049FFEF73EFF2B68019A1C121340D54A25
:101820009B009B58049F0435FEF764FF039A3B1D01
:101830000493D14C9B1ADB2B04DD1A23009E2370EA
:10184000FEF727FF01F04AFDCC4B40001840012372
:10185000184323783860002B03D0009E049FFEF7C6
:1018600018FF2B68019A1C121340C24A9B009B5818
:10187000049F0435FEF73EFFA4003E1B3000FEF738
:10188000E5FDBD4B30601B78371D002B02D0009E5C
:10189000FEF7FFFE2B68019A1C121340B54A9B000D
:1018A0009B580435FEF726FFA4003F1B3800FEF7C7
:1018B000E5FDB14B1B78002B02D0009EFEF7E9FE40
:1018C0002B68019A1C121340AA4A9B009B580435AE
:1018D000FEF710FFA300FB1A0493012320001A0057
:1018E0000499FEF71FFEA64C2068643001F044F80E
:1018F000002816D0029B21685A78A24801F0BBFA52
:1019000015E0A300FB1A0493200001230022049990
:10191000FEF708FE9A4C2068643001F02DF800288C
:1019200002D1043DFEF7C9FE964801F03FF90123BC
:10193000029A137001F0D2FCC8222368D200063349
:1019400053431818029B5860FEF7B8FEFEF762FE7C
:10195000894BA4001B783E1B3060371D002B02D042
:10196000009EFEF796FE2B68019A1C121340814AD6
:101970009B009B580435FEF7BDFEA4003E1B3000C3
:1019800001F0EAFC7C4B30601B78371D002B02D045
:10199000009EFEF77EFE2B68019A1C121340754ACA
:1019A0009B009B580435FEF7A5FEA4003E1B3000AB
:1019B00001F0D4FC704B30601B78371D002B02D037
:1019C000009EFEF766FE2B68019A1C121340694ABE
:1019D0009B009B580435FEF78DFEA4003E1B300093
:1019E00001F0BEFC644B30601B78371D002B02D029
:1019F000009EFEF74EFE2B68019A1C1213405D4AB2
:101A00009B009B580435FEF775FEA4003F1B380071
:101A100001F0C4FC584B1B78002B02D0009EFEF74F
:101A200038FE2B68019A1C121340524A9B009B58A7
:101A30000435FEF75FFEA4003E1B300001F0D0FC31
:101A40004D4B30601B78371D002B02D0009EFEF7F7
:101A500020FE2B68019A1C121340464A9B009B589B
:101A60000435FEF747FEA4003F1B380001F0EAFCF6
:101A7000414B1B78002B02D0009EFEF70AFE2B681C
:101A8000019A1C1213403B4A9B009B580435FEF7F9
:101A900031FE0121200001F0BDFC374B1B78002BEB
:101AA00002D0009EFEF7F5FD2B68019A1C12134030
:101AB000304A9B009B580435FEF71CFE0021200095
:101AC00001F0A8FC2C4B1B78002B02D0009EFEF7E7
:101AD000E0FD2B68019A1C121340264A9B009B587C
:101AE0000435FEF707FEA4003E1B300001F0C8FCE1
:101AF000214B30601B78371D002B02D0009EFEF773
:101B0000C8FD2B68019A1C1213401A4A9B009B586F
:101B10000435FEF7EFFDA4003E1B300001F0C4FCCD
:101B2000154B30601B78371D002B02D0009EFEF74E
:101B3000B0FD2B68019A1C1213400E4A9B009B5863
:101B40000435FEF7D7FDA4003F1B380001F086FCEA
:101B5000094B1B78002B02D0009EFEF79AFD2B68E4
:101B6000019A1C121340034A9B009B580435FEF750
:101B7000C1FDC046E467000030020020FEFFFF7F89
:101B8000380200203C020020A4003F1B380002F075
:101B900071F9D84B1B78002B02D0009EFEF779FD1F
:101BA0002B68019A1C121340D34A9B009B580435A2
:101BB000FEF7A0FDA4003E1B300002F0CBF9CD4B98
:101BC00030601B78371D002B02D0009EFEF761FDB0
:101BD0002B68019A1C121340C74A9B009B5804357E
:101BE000FEF788FDA4003F1B380002F013F9C14B3B
:101BF0001B78002B02D0009EFEF74BFD2B68019A4C
:101C00001C121340BC4A9B009B580435FEF772FD22
:101C1000A4003E1B300002F013F9B64B30601B7875
:101C2000371D002B02D0009EFEF733FD2B68019A72
:101C30001C121340B04A9B009B580435FEF75AFD16
:101C4000A4003F1B380001F01FFFAA4B1B78002B9C
:101C500002D0009EFEF71DFD2B68019A1C12134056
:101C6000A54A9B009B580435FEF744FDA4003F1B8A
:101C7000380001F01FFF9F4B1B78002B02D0009E05
:101C8000FEF707FD2B68019A1C1213409A4A9B002D
:101C90009B580435FEF72EFDA4003F1B380001F0D1
:101CA00019FF944B1B78002B02D0009EFEF7F1FC2D
:101CB0002B68019A1C1213408F4A9B009B580435D5
:101CC000FEF718FDA4003F1B380001F02BFF894BE5
:101CD0001B78002B02D0009EFEF7DBFC2B68019ADC
:101CE0001C121340844A9B009B580435FEF702FDEA
:101CF000A300FE1A31002000049302F06CF9049B4B
:101D00003060FF1A7B4B04371B78002B02D0009EFB
:101D1000FEF7BFFC2B68019A1C121340764A9B0009
:101D20009B580435FEF7E6FCA300FE1A31002000A4
:101D3000049302F068F9049B3060FF1A6D4B04377E
:101D40001B78002B02D0009EFEF7A3FC2B68019AA3
:101D50001C121340684A9B009B580435FEF7CAFCCE
:101D6000A300FE1A31002000049302F00EF9049B38
:101D70003060FF1A5F4B04371B78002B02D0009EA7
:101D8000FEF787FC2B68019A1C1213405A4A9B00ED
:101D90009B580435FEF7AEFCA300FE1A310020006C
:101DA000049302F00BF9049B3060FF1A514B043787
:101DB0001B78002B02D0009EFEF76BFC2B68019A6B
:101DC0001C1213404C4A9B009B580435FEF792FCB2
:101DD000A4003F1B380001F0CDFE464B1B78002BC2
:101DE00002D0009EFEF755FC2B68019A1C1213408E
:101DF000414A9B009B580435FEF77CFCA300FF1A68
:101E00003900200001F06CFF3A4B1B78002B02D008
:101E1000009EFEF73EFC2B68019A1C121340364AC6
:101E20009B009B580435FEF765FCA4003E1B300068
:101E300001F022FF2F4B30601B78371D002B02D0A2
:101E4000009EFEF726FC2B68019A1C1213402A4ABA
:101E50009B009B580435FEF74DFCA300FF1A390088
:101E6000200001F0E7FE234B1B78002B02D0009EE0
:101E7000FEF70FFC2B68019A1C1213401E4A9B00B0
:101E80009B580435FEF736FCA300FF1A39002000EA
:101E900000F0F6FC174B1B78002B02D0009EFEF7DB
:101EA000F8FB2B68019A1C121340134A9B009B58A5
:101EB0000435FEF71FFCA300FE1A31002000049336
:101EC00000F0DEFC049B3060FF1A0A4B04371B78DD
:101ED000002B02D0009EFEF7DCFB2B68019A1C123F
:101EE0001340054A9B009B580435FEF703FC07B0DE
:101EF000F0BDC04630020020E46700000023F7B5C3
:101F00005A1E0192002B07DA01F06AFC00F024FF50
:101F100000F0D6FF6423019300263000194B1968A6
:101F20008E4201DB019BEBE7174B1A6801329142AD
:101F300000DC0022F0241A601D68144F6C43E35D3E
:101F4000002B1DD0E419022B16D0012B0ED1002836
:101F500001D101F0C3F9F0226A430C4B0C499B18E4
:101F60005B68C31A8B4201D80223BB54F0235D4344
:101F7000064BEB5C022B03D12000FEF763FBD1E79D
:101F80000136CBE73402002000000020441100207D
:101F90009F860100054B01211A68054B1A6000233A
:101FA000044AD1500433642BFBD1704788050020CC
:101FB000800500209C22002000B59BB0020005494E
:101FC00001A803F05FFD01A800F00CFE00F078FF0F
:101FD000FCE7C046246A000037B5174D04002868A6
:101FE000002801D003F042F9A400200003F034F9E6
:101FF0002860002801D1114809E001AB984208D2BD
:102000000F4B02196B440193934202D20D48FFF724
:10201000D3FF042802D808302860083C2B680A4AFD
:102020001C191360094B01211C600023084AD15080
:102030000433642BFBD137BD88050020356A0000CE
:102040001CFCFFFF656A000080050020840500205D
:102050009C22002070B50D4D0D4E2B684C1CA40029
:1020600036681C19B44203D90A20FEF7CDFA0BE0FA
:102070002C601D00AC4201D904C5FBE70F22090109
:10208000104008431860180070BDC046800500204D
:10209000840500200322CB1C70B50C00D917114019
:1020A000C9180500891000220420FFF7D3FF002380
:1020B000A34204DAE95CC21811710133F8E7E14385
:1020C0000023C917214041180B7170BD10B583075B
:1020D00006D1042804D90F2304C81340042B03D0CD
:1020E0000E20FEF791FA014810BDC0466C6B00004F
:1020F00030B502248025094B094AED009C505C59FB
:10210000002CFCD0A124E400884204D28025ED00FC
:1021100018514019F8E70021995030BD00E0014006
:102120000405000010B5002804D19020922100027F
:10213000890203E0922080218002C902FFF7D8FFC4
:1021400010BD002802D092239B0201E090231B02C5
:102150001B6800201A0E532A01D11B02180A70476F
:1021600030B501248025064A064BED00D450545961
:10217000002CFCD001600021014AD15030BDC04686
:1021800000E001400405000010B5002802D09220B4
:10219000800201E090200002A6230902DB05090A63
:1021A0001943FFF7DDFF10BDF0B5012480250300C2
:1021B0000F4F08000F49ED007C507C59002CFCD0DB
:1021C0009C46002810DD5478167893782402344316
:1021D0001B0423431C00D37801381B0623436446A9
:1021E00008C40432A446ECE700237B50F0BDC0468F
:1021F00000E001400405000070B505004B680A00CE
:102200009C1C2100FFF7D0FFA000281870BD000023
:10221000154B1B68002B04D080219223C9029B021E
:1022200003E09221902389021B02002807D1191D87
:102230005B6802001B0E522B14D10A0012E0002230
:1022400081420FD903681B0E522B0BD14368023316
:102250009B00C318994205D91A68110E0022522911
:1022600000D11A00100070478C0700208022F0B5C2
:10227000520085B00021624803F00BF88022002153
:102280005200604803F005F85F4B1B681A00029388
:1022900053425A4110000392FFF744FF029B002B68
:1022A00001D15A4C00E05A4C0020FFF7B1FFFF2744
:1022B0000500002D00D194E02B681A121B143A403F
:1022C0003B4001921A000A3A092A43D84C4B019A22
:1022D000995C002900D07FE010224E4802F0D9FF1F
:1022E0002E00336801991A123A40914217D11A14FC
:1022F0003A400B2A06D0132A0CD00A2A0FD1454B9C
:102300001E600CE03B40022B09DC424A9B00D318C4
:102310005E6004E0102200213E4802F0BAFF300067
:10232000FFF776FF061EDCD13A4B196800290FD063
:102330002000FFF761FF0400374E3168002903D009
:102340002000FFF759FF0400344B0436B342F4D1A8
:102350002B4B3EE0143B092B3ED82A4B019A995C4B
:10236000002939D108222E4802F093FF2E0033684D
:102370001A143A40152A0BD01D2A11D0142A14D150
:10238000019A1B123B409A420FD1254B1E600CE074
:10239000019A1B123B409A4207D1214B5E6004E038
:1023A000082200211E4802F074FF3000FFF730FFC2
:1023B000061EDCD11A4E3168002909D02000FFF733
:1023C0001BFF71680400002902D0FFF715FF04000D
:1023D0000C4B0121019A99542800FFF719FF0500C1
:1023E00067E70298FFF7ADFE411C0398FFF7CCFEAC
:1023F000054B039A1A600B4B1C6005B0F0BDC0463C
:102400008C0600208C0500208C0700200448020068
:10241000049000000023002004230020102300204B
:10242000102300209007002070B50020FFF789FEE0
:1024300004000120FFF785FE844200DA04000A4B05
:102440001E687542754128001D60FFF76BFE002E67
:1024500001D0064B00E0064B064A2800611C1360C1
:10246000FFF792FE70BDC0468C070020049000006C
:102470000448020090070020F8B50020FFF761FE35
:1024800007000120FFF75DFE3E00224D0643224C6F
:102490000CD180219020C9020002FFF729FE012102
:1024A0003000FFF771FE2E601C4B2FE0874208DDE5
:1024B000002392212B60194B89022360236800209E
:1024C00011E0012380212B60154BC9022360F5E741
:1024D0001A68551C18D0120E522A07D101205A68CA
:1024E000023292009B188B42F2D311E0002800D0F8
:1024F00023600C4C0C49200003F0F0FA200000F09F
:10250000FFFEFFF791FF04E0002802D0236000E007
:102510002160F8BD8C070020900700200490000087
:102520000448020054230020DD6A0000F0B585B0A5
:10253000039203220333DC1714402A4EE3189C1045
:10254000336801900291002B02D08022D20201E078
:1025500092229202244FA51C3B68AD005B199A425F
:1025600017D2FFF783FE3368002B02D08022D202FD
:1025700001E0922292023B685B199A4209D21B4CFD
:102580001B49200003F0AAFA200000F0B9FE002049
:1025900026E0029B3E681B06190C6B461A7BA4239F
:1025A000DB051343019A0B431104FF22120411406F
:1025B00019433000FFF7D4FD3300301D08332100EC
:1025C00001933B60FFF7CCFD002C04D00A9A210058
:1025D0000198FFF7E9FD3000019B083D5D193D6062
:1025E00005B0F0BD8C070020900700205423002088
:1025F000066B000070B59AB0FFF73EFFFF221F4C3C
:10260000D2000021200002F044FE0020FFF700FE6F
:10261000FF25002600281AD003681A142A400A2A27
:1026200008D11A122A40FF2A0ED0D200A1180B712D
:10263000A05009E0132A07D11B122B40FF2B03D017
:10264000DB00E2181671E650FFF7E2FDE2E7FF213A
:102650000200C900235808305D1EAB41D2188842E1
:10266000F8D1074901A803F00DFA01A800F0BAFA61
:10267000044800F0B7FA1AB070BDC046A41A002092
:102680002D6B0000456B0000002070470120704753
:10269000004870473C2300200048704733F8FFFF94
:1026A00010B50449044803F019FA242303480360D1
:1026B00010BDC046006C00001C2300201823002021
:1026C00000207047002070470020704700207047AE
:1026D000002070470020704700207047002070479E
:1026E0000020704710B5034A0E21034800F0B4F8EB
:1026F00010BDC04604000020056C0000044A0549D6
:102700001368C85401339B059B0D13607047C04686
:10271000980B002094070020114A70B51368114CE3
:10272000984211DA015D451CFA39012906D8AB42FD
:1027300006DD2118497801391F2901D92800EFE762
:102740000100251A461C02D10023136006E0665CD6
:102750006E5401318B42FADC181A106070BDC0460D
:102760009C0B0020A40B002010B500F0B7FD064B19
:102770001A68904201D200221A601B68C01A034BEB
:1027800083428041404210BDA00B0020204E00003B
:1027900010B5094C094A2368126893420BD0084AC5
:1027A000D05C00F0D7FE002805D0236801339B05DC
:1027B0009B0D2360EDE710BDA40F0020980B0020B7
:1027C0009407002010B50400064B074A1B681268E6
:1027D0009B1ADB439B059B0DA34202DAFFF7D8FF50
:1027E000F2E710BD980B0020A40F0020F7B50600FB
:1027F0000191151E2FD05768B800441C0630FFF712
:10280000E1FFFB20FFF77AFF1C20FFF777FFF0B214
:10281000FFF774FFE0B22412FFF770FFE0B2FFF79A
:102820006DFF6B461879FFF769FF0026BE4212DA8A
:10283000B300EB189C680136E0B2FFF75FFF20128F
:10284000C0B2FFF75BFF2014C0B2FFF757FF200EA6
:10285000FFF754FFEAE7F7BD70B5074D2C68092C68
:1028600008DC0C236343054E01349851F31859607A
:102870009A602C6070BDC046A80F0020B8230020CD
:10288000F0B589B004900E0001284BDD284B086894
:102890000293830709D1042807D90F230268134044
:1028A000042B02D1FFF712FC0290214B70680393B6
:1028B000830709D1042807D90F2302681340042B8A
:1028C00002D1FFF703FC039000271A4B1A4D1B6837
:1028D0000593059B9F4225DA2B1F0299186803F088
:1028E000F3F800281BD12B686C6806930190019BBC
:1028F000069A934213DA20680399079403F0E4F8E8
:102900000834002807D131000498079B08315B6820
:102910000238984709E0019B01330193E7E701374B
:102920000C35D6E71B20FDF76FFE09B0F0BDC046A1
:102930006C6B0000A80F0020BC23002010B501F034
:1029400043FA00F0C7FD00F033FEFFF7CBFE01F0C5
:1029500085FA01F083FB10BD962210B5120100210B
:10296000034802F096FC0022024B1A6010BDC046DC
:102970004411002034020020064B074A1B681268ED
:102980009B1ADB439B059B0D0122834200DC002246
:1029900010007047980B0020A40F0020F8B5050028
:1029A0000C0016001F1E0ED10320FFF7E5FF0028C4
:1029B00027D0FA20FFF7A2FEE8B2FFF79FFEE0B2B1
:1029C000FFF79CFE1DE0501DFFF7D6FF002818D032
:1029D000FB20FFF793FEE8B2FFF790FEE0B2FFF7AF
:1029E0008DFEF0B2FFF78AFE3012C0B2FFF786FE0E
:1029F0003C00E31B9E4204DD2078FFF77FFE01349C
:102A0000F7E7F8BD70B50024F0250B4B1B689C421E
:102A10000EDA2A006243094BD3181A78002A05D02F
:102A20005978002311201A00FFF7B8FF0134ECE7B2
:102A3000FFF792FF70BDC046340200204411002011
:102A40000123F3B50400FFB00D0010001A420DD0B1
:102A500002AA1370431002A9537042121B0E4014B5
:102A60008A700B71C8700B00052273E003231340BA
:102A70001ED1042A1CD90F2201680A40042A17D14A
:102A8000023302AA1370FFF721FB060003F02EF8B1
:102A9000F823FF33984200DD18000023834205DA53
:102AA00001335A1EB25C02A9CA54F7E7421C50E037
:102AB000042801D0002809D1032302AA0438137086
:102AC0004342434153701300022243E0002B45D19F
:102AD000042843D90F2102681140052912D104337B
:102AE00002A90B70F8231209FF3392009A4200DD0D
:102AF0001A00002393422BDA0133C118C97802AEC1
:102B0000F154F7E7062929D101390E00120956437D
:102B10000196F826019FFF36B7421FDC02AE3170E6
:102B20000136934213DA01270133990041583942A3
:102B300001D0394100E00A49012737700F12717046
:102B4000B7700F14090EF77031710536E9E7019A75
:102B5000013202AB29002000FFF720FF7FB0F3BD58
:102B600019FCFFFF70B5F023050000240D4A180082
:102B7000604380184178A94203D001340A2CF6D171
:102B80000FE0F022002102F084FB074A1368013BAA
:102B9000A34200D11460002329001A001120FFF77E
:102BA000FDFE70BD441100203402002010B5B2B00B
:102BB00002236A460400137002F098FFC72800DD64
:102BC000C7200023834205DA694601335A1EA25CFE
:102BD000CA54F7E7421C6B46FE211420FFF7DEFEC5
:102BE00032B010BD10B5B2B002236A4604001370B3
:102BF00002F07CFFC72800DDC7200023834205DAEE
:102C0000694601335A1EA25CCA54F7E7421C6B4660
:102C1000FF211420FFF7C2FE32B010BDF7B5234BE1
:102C200006001B68F020009300232149009A93427C
:102C30000ADA02005A438A185478B44202D1127850
:102C4000002A31D10133F1E70024F0231A00624356
:102C500001920199164A55182F78002F06D0013499
:102C60000A2CF3D11348FFF7BDFF1DE0F022390015
:102C7000280002F00EFB02230D4A0199EB60535429
:102C80000D4AF1008A58009B6E70AE70AA602F61E9
:102C90006F61A34202DC054B01341C60002331004C
:102CA0001A001020FFF77AFEF7BDC046340200205C
:102CB00044110020C06C0000A41A002010B5FFF7DA
:102CC000A1FE0024064BE200D3181B79043B012B24
:102CD00002D8E0B2FFF7A2FF0134FF2CF2D110BD01
:102CE000A41A0020F7B50E0000247F250190194B8F
:102CF000E200D1180979062901D0032926D1985874
:102D000083682B401C2B21D1C3681A002A40042A57
:102D10001CD102692A40192A18D11B0A01339B00D1
:102D20000C30C018FFF7D2F9070002F0DFFE0023D5
:102D3000B0420BD19E4206DD019AF95CD25C914211
:102D400004D10133F6E7E0B2FFF768FF0134FF2C4E
:102D5000CDD1F7BDA41A002070B500F0BFFA184B12
:102D60001A68904201D200221A601A681549821A24
:102D70008A4223D91860002000F082FB444244417B
:102D8000604207240443002000F08EFB002810D08E
:102D9000082600250C4BEA00D3181B799C4201D071
:102DA000B34202D1E8B2FFF739FF0135FF2DF1D16F
:102DB00004E0631C02D001267642EAE770BDC046FB
:102DC000940B00200F270000A41A002037B5002420
:102DD0000500FFF717FE01A8019400F03FFB20005B
:102DE00000F068FE00F0FCFC00F072FB00F071FBEC
:102DF00000F038FF00F09EFA0548FFF7F3FEA54209
:102E000004D0FFF7C7F80348FFF7ECFE37BDC04614
:102E1000D56C0000ED6C0000002310B501001A0015
:102E20001120FFF7BBFD10BD07B56B461970694651
:102E30005A7013128B701314120ECB700A716B46FA
:102E4000010005221320FFF7A9FD07BD10B50A00F8
:102E500001001220FFF7F4FD10BD70B50500080059
:102E60000C003230FFF7AEFC2B00220000211B20AB
:102E7000FFF794FD70BD10B50C0003001100142085
:102E80002200FFF78BFD10BD70B506000020FFF794
:102E9000BFF90024FF25002810D003681A142A4027
:102EA000152A05D11B122B40B34204D1040002E0C5
:102EB0001D2A00D10024FFF7ABF9ECE7200070BD1C
:102EC000F0B580279DB0FFF763FCB94DB94C286879
:102ED000FF00391A201800F023FB2B680600C318E6
:102EE0002B60002B00D1DBE1002E0DDD2868391AA4
:102EF000201800F015FB2B6806001B182B6000F053
:102F0000EDF9AD4B1860EFE72378FA2B00D00CE118
:102F10002B68022B06DCFFF727FC002800D1BFE15D
:102F20000120B8E16078A5780238182800D9FAE0C5
:102F300001F07AFF0D1E22262932F93D676F75894F
:102F4000DAEFF9F9F9F9F9F9F9F9F9F9F300FF2DDF
:102F500000D1E8E02800FFF705FE00229749EB00CA
:102F60005A50CB181A7129000092130013204DE01B
:102F70002800FFF753FED6E02800FFF7F3FDD2E06C
:102F8000FFF79CFECFE0FFF73DFD0020FFF71EFF9F
:102F90008B48FFF727FEC6E0182D00D9C3E0894B08
:102FA000AA00D25829001520FFF74AFDBBE00024F3
:102FB0002000FFF769FF071E03D10134192CF7D158
:102FC000B1E0083002F092FD06000530FFF7FAFB91
:102FD000FB20FFF793FB1D20FFF790FBE0B2FFF70C
:102FE0008DFBF0B2FFF78AFB3012C0B2FFF786FB11
:102FF0000025AE42E1DD7B19187AFFF77FFB013532
:10300000F7E700211D200B000A000091FFF78EFA60
:1030100089E000222900009213002720F6E700F043
:1030200077F903AC684A64210090684B200002F0F5
:10303000F7FC02232000237002F058FD2300020059
:10304000002116206DE000245C4AE300D558002DD5
:1030500046D06B689E00701DFFF7B4FB2B00002567
:103060003200083321000120FFF798FC0020FFF711
:10307000CFF82E002F0000281DD0FF2103681A1260
:103080000A40A24214D11A140A400B2A07D10B405D
:103090000DD0012B09D0022B00D1FFE008E0132A4C
:1030A00006D100252E002F0002E0060000E00700F8
:1030B000FFF7AEF8DFE7002E04D032000121200038
:1030C000FFF794FB002D04D02A0002212000FFF717
:1030D0008DFB002F04D03A0000212000FFF786FB73
:1030E0000134FF2CB0D11EE0FFF78CFC002500243A
:1030F000290000942300220013200135FFF716FA5F
:10310000FF2DF4D1FF222100D2002C4802F0C1F89B
:1031100009E00120FFF75AFE05E0002329001A000C
:103120001A20FFF73BFC0320B5E0FB2B00D0F7E6AD
:103130002A68042A00DCEEE62679E078244B360281
:1031400006439E4200DDEBE6331D9A4200DCE2E6D8
:10315000E35CFE2B00D0E3E66078A578731E1C28A4
:1031600068D007D8082835D01B285ED0012800D0A9
:1031700090E007E01E2800D17EE066D31F2800D132
:1031800080E087E0FF2D00D184E02800FFF7EAFC13
:1031900067790634B31E290000943A000A20FFF72D
:1031A000C5F9064BED00E8505D192F7172E0C0467D
:1031B0009C0B0020A40B0020A00B0020A41A0020D0
:1031C000FD6C00009C220020146D00000F6D0000BB
:1031D000F6030000182D5DD86079022813D003286B
:1031E0001BD0012856D1A71D7A78A479BB7812028A
:1031F00022431B0413431A00FB78AD001B06134344
:103200005B0003430EE0002B44DDB11EA01DFEF762
:1032100041FF244BAD00E8503CE0A379AD005A1EBD
:1032200093419B001F4AAB5034E0601D1900FFF72B
:1032300059FD2FE0FF2D2DD06279022A2AD80634BD
:10324000B31E009429000B2022E0632B00DD6323D2
:10325000002203A8934204DDA11849798154013268
:10326000F7E7D9430022C917194041180A70013302
:103270000090290015200BE005340094002229005D
:103280001E2005E0042B05D10022290005340094FE
:10329000FFF74CF9701DFFF73FFA01E0050007E763
:1032A0001DB0F0BD9C220020002070470020704718
:1032B000002070470020704701220020054B06497E
:1032C0001A61585003300431585080180831585052
:1032D0001A60704700800040040500000122034B83
:1032E0001A64A822D20098587047C0460080004057
:1032F00010B5FFF7F3FFFA21890001F09FFD10BD23
:1033000010B50100014801F043FB10BDD0100020B2
:1033100000487047246D000070B5054E0400335C12
:103320000D008B4202D001F05BFA355570BDC046EE
:10333000AC0F002070B50024064D635D012B05D154
:103340000021200001F04CFA0023635501341A2CAF
:10335000F2D170BDAC0F00200D20704735207047B2
:10336000036870B55B100120052B12D8094A9B0039
:103370009C58094D2B5D002B05D00021200001F049
:103380002FFA00232B55200001F0D4F80123400030
:10339000184370BD506D0000AC0F002070B503687D
:1033A00045685C106D1004D40B4B9D4202DD1D007E
:1033B00000E00025192C0DD8084E335D012B05D0F7
:1033C0000121200001F00CFA0123335529002000CF
:1033D00001F03EF970BDC046FF030000AC0F0020B5
:1033E00070B504686410192C0FD8094D2B5D002BA3
:1033F00005D00021200001F0F3F900232B55200017
:1034000001F022FA0423012800D00023180070BD27
:10341000AC0F002070B504000D0019280ED8084E1E
:10342000335C012B04D0012101F0DAF9012333557B
:10343000290020004D1EA94101F0F0F970BDC046E1
:10344000AC0F0020436810B5191F4A424A4100687A
:1034500011004010FFF7DEFF10BD000037B56946D0
:103460000200064B684630CB30C11368042B02D1F2
:1034700000F030FB01E000F055FB37BD1C6D000093
:1034800010B5084C237D002B05D00021142001F03D
:10349000A7F900232375142001F0D6F943425841BF
:1034A000800010BDAC0F002010B5084CA37D002B90
:1034B00005D00021162001F093F90023A3751620F2
:1034C00001F0C2F943425841800010BDAC0F00200A
:1034D0007047704710B5034A04210348FFF7BCF951
:1034E00010BDC04674000020156C0000E12110B52D
:1034F0004902094801F093FAFFF7DEFE0A2001F0C5
:1035000013F80023FF21054A995401331A2BFBD1EC
:1035100000F0A8FB10BDC046D0100020AC0F00206A
:10352000F8B50B4E070030000D0001F0B7FA041E8D
:10353000AC4200DD2C003D00EB1B9C4205DD300061
:1035400001F0B6FA28700135F6E72000F8BDC04654
:10355000D010002010B50100014801F067FA10BD3D
:10356000D01000200020704710B51E20FDF74CF849
:1035700010BD10B51E20FDF747F810BD10B51E2078
:10358000FDF742F8002010BD10B51E20FDF73CF8F5
:1035900010BD10B51E20FDF737F810BD10B51E2068
:1035A000FDF732F810BD10B51E20FDF72DF810BD47
:1035B00010B5034A08210348FFF74EF910BDC04675
:1035C00094000020686D00000123034A1360034A41
:1035D0001068984018437047D00F0020D80F002083
:1035E0001E2800D91A20084B8000C258012393409E
:1035F000064A07491360074A1160074A07491160E4
:10360000074A13607047C04630720000CC0F00209C
:1036100008050050E80F0020E00F00200C050050C6
:1036200018050050F0B5EFF310810123194083F322
:103630001088134E134AB4461268013A9340124A56
:103640001468124A1568124A002B15D016680342F6
:103650000BD02660C046C046C046C046C046C046E5
:10366000C046C04616682E6004E067463E60166895
:10367000084F3E605B08E7E781F31088F0BDC04665
:1036800008050050DC000020E80F0020E00F0020BB
:10369000CC0F00200C05005030B585B001AD0C22D8
:1036A0000649280001F0ECFD0024285D01210134C9
:1036B000FFF732FE0C2CF8D105B030BDDE6D0000F6
:1036C000F0B53B4C85B0210003220C31684601F077
:1036D000D7FD210009220F3101A801F0D1FDFFF72C
:1036E00007FE344B344CC0182368984201D20023A3
:1036F00023602568002D3ED12E006B4604339F5D6C
:1037000001213800FFF708FE01360121380001F0E1
:1037100085F8092EF1D100266B469F5D0121380006
:10372000FFF7FAFD01360021380001F077F8032E8B
:10373000F2D1C82080000138C046C046C046C0460D
:10374000C046C046C046C046C046C046C046C04649
:10375000F1D100210520FFF7DFFD00266B46002197
:10376000985D0136FFF7D8FD032EF7D1FFF7C0FDB6
:103770001330206019E0FFF7BBFD23680025984255
:1037800013D3052000F0D6FE0C4B0D4EC01801D40B
:10379000306000E035603068032101F0D9FB002380
:1037A0000125084A306023601360280005B0F0BD91
:1037B000DE6D000010270000C80F0020C8FEFFFFCC
:1037C000D80F0020D00F002010B50124044001D0F4
:1037D000441002E00D20FCF717FF200010BD000090
:1037E0007FB5A44E3368002B0BD1A34A1268002A80
:1037F00007D1A24B1B68002B00D139E1FFF760FF16
:1038000036E19F4D2A68002A2AD19C4A1268002A74
:1038100007D0FFF755FF002800D129E1FFF73CFF53
:1038200005E0954A1268002A01D1002BF6D1924B8F
:1038300019681A00002911D03468002C0ED101AD8E
:103840000C22904928001C6001F01AFD285D00211F
:103850000134FFF761FD0C2CF8D109E133681360E6
:1038600000210D2000F0DAFF00210E2000F0D6FF2D
:1038700000210F2000F0D2FF2E68012E56D0022E1C
:1038800000D19CE0002E00D0ECE0013631007A4CF3
:1038900004202368994300F0C1FF04212368052018
:1038A0000B405942594100F0B9FF1021236806200E
:1038B0000B405942594100F0B1FF802123680901B2
:1038C0000B40594259410C2000F0A8FF8021236889
:1038D00009020B40594259410B2000F09FFF802103
:1038E000236849020B40594259410A2000F096FFD3
:1038F0008021236889020B4059425941092000F078
:103900008DFF80212368C9020B405942594108208C
:1039100000F084FF802321681B030B40594259416A
:10392000072000F07BFF31000D2099E00221524C6E
:10393000072023680B405942594100F06FFF0820CF
:10394000216801400B005942594100F067FF802176
:103950002368C9000B4059425941052000F05EFF21
:103960008021236849010B4059425941062000F04B
:1039700055FF80212368C9010B4059425941042059
:1039800000F04CFF8021236889030B4059425941C4
:103990000A2000F043FF802321681B040B4059429A
:1039A0005941092000F03AFF31000C2000F036FFA9
:1039B00031000B2000F032FF31000E2050E02021BA
:1039C0002D4C072023680B405942594100F026FF37
:1039D0004021236808200B405942594100F01EFF46
:1039E0008021236809200B405942594100F016FFFD
:1039F0008021236849000B40594259410A2000F0B8
:103A00000DFF8021236889000B40594259410B204A
:103A100000F004FF8021236889010B40594259417D
:103A20000C2000F0FBFE8021236849030B40594223
:103A30005941062000F0F2FE80212368C9030B40A3
:103A400059425941042000F0E9FE802321685B04BB
:103A50000B4059425941052000F0E0FE01210F20A2
:103A600000F0DCFE2B680321581C01F057FB296095
:103A70007FBDC046DC0F0020D40F0020D00F0020F7
:103A8000E40F0020DE6D0000006810B5C30703D509
:103A9000FFF79AFE054B1860054B1B68002B03D0FF
:103AA000024B186800F0D9FA10BDC046DC0F0020A8
:103AB000F00F00200022054B10B51A60044B1B6864
:103AC000934201D000F0C7FA10BDC046DC0F0020C1
:103AD000F00F002070B505000068FFF775FE0400C8
:103AE0006868FFF771FE631E0100042B14D8451EA1
:103AF000042D11D805226A43D318012215009D40D8
:103B00002B00064805682B430360054B1B68002B00
:103B100002D0200000F0A0FA70BDC046DC0F0020EB
:103B2000F00F002070B505000068FFF74DFE04009F
:103B30006868FFF749FE631E0100042B14D8451E78
:103B4000042D11D805226A43D31801229A4013008C
:103B5000064802689A43064B02601B68002B03D09C
:103B60000022200000F078FA70BDC046DC0F002073
:103B7000F00F00202C4BF7B51B680400002B03D17D
:103B800001204042FFF72CFD01262468344219D061
:103B9000FF226310180212041040FF226112120269
:103BA0000A40DBB210431843204B1B68202B06D180
:103BB000B4401F4BA40EA400E35800021843FFF7C3
:103BC00031FD30E0032525402DD1042C2BD90F23C6
:103BD00022681340062B26D1FF27130901933F04C7
:103BE000019B9D421FDAAB00E3185A68324218D09D
:103BF000531018023840FF21844609025012084031
:103C00006146DBB208431843084B1B68202B06D1E2
:103C10005200920E064B9200D35800021843FFF751
:103C200001FD0135DCE7F7BDCC0F0020DC000020F2
:103C30000C6E00000B6810B50200D80701D55810B3
:103C400001E0012040421823012A03DD4A68042ACA
:103C500000D10833024A1360FFF7C2FC10BDC04612
:103C6000DC000020012010B54042FFF7B9FC002025
:103C7000FFF7D8FC10BD00000068F8B5C30702D5F7
:103C8000FFF7A2FD0BE0830726D1042824D90F22D9
:103C900003681A40042A1FD11B091DD000790300B4
:103CA000203B5E2B18D80522002053430B4E9D1855
:103CB000043AAB420CD0052110249F5D3C4200D059
:103CC00080180139520064100029F7D10133F0E760
:103CD00001234000184300E00120F8BD0C6F0000F4
:103CE000F0B5050085B008680C00FFF76DFD039086
:103CF000022D08DD6068FFF767FD0700A068FFF789
:103D000063FD040001E00124270005236343053B14
:103D10000293012326000193231D9E4234DC3D00C3
:103D20003B1D9D422BDC731E042B23D86B1E042BE2
:103D300020D8029B039A591E019B49191A40204B17
:103D40000AD001228A4019680A431A601D4B0122D9
:103D50001B68002B0ED009E0012088400100186884
:103D600088431860174B1B68002B03D031002800D4
:103D700000F072F9019B01355B000193D0E7029BD3
:103D8000013605330293C7E73D1D042D15D8012CDC
:103D900013D126003300AB40094A11689943094BFF
:103DA00011601B68002B04D0781D0022210000F058
:103DB00053F901340535062CECD105B0F0BDC046F1
:103DC000DC0F0020F00F002010B5034A012103484A
:103DD000FEF742FD10BDC046D4000020F66D000085
:103DE0000120704710B501210D20FFF795FA012140
:103DF0000E20FFF791FA00210F20FFF78DFA044CF7
:103E0000200000F09DF91021200000F0B5F910BD50
:103E10000010002010B504680D20E30703D56410DE
:103E2000FF2C03D91720FCF7EFFB06E0FFF7DAFFC2
:103E3000E1B2024800F0C2F9002010BD00100020DD
:103E400010B5FFF7CFFF0021034800F0B7F90123B9
:103E50004000184310BDC0460010002010B5034AB2
:103E600005210348FEF7F8FC10BDC046E000002025
:103E7000E7700000F7B501260468344205D04268B7
:103E8000324202D08368334201D10D2005E0521046
:103E900064100092802C03D91520FCF7B5FB23E0B9
:103EA000009A1620FF2AF8D85B1001931720FF2BE9
:103EB000F3D80E4F0E4D3B68002B03D1280000F0C5
:103EC00003FA3E60E1B2280000F08CFA6B4628004D
:103ED000197800F0BAF96B462800197900F0B5F9A5
:103EE000280000F0E9FA0020FEBDC046EC0F0020DB
:103EF00014100020F8B5154F05003B680E00144C57
:103F0000002B04D1200000F0DFF901233B60EDB26B
:103F10002900200000F066FAF1B2200000F095F9C7
:103F20000021200000F06AFA002801D040420CE095
:103F300001222900200000F050FA200000F07BF957
:103F40000028FAD0200000F07BF9F8BDEC0F00202B
:103F50001410002010B501240368234202D04168E8
:103F6000214201D10D2004E058104910802803D9C6
:103F70001520FCF749FB07E0FF2901D91620F8E7D7
:103F8000FFF7B8FF4000204310BD10B507211820EF
:103F9000FFF7B0FF7F2801DD0138FF3803007F33D2
:103FA00001DA7F20404264237F215843494200F0D8
:103FB000CFFF012340424000184310BD10B5082137
:103FC0001820FFF797FFC30F181801234010153072
:103FD0004000184310BD10B505211820FFF78AFFD7
:103FE0007F2801DD0138FF3803007F3301DA7F20AD
:103FF000404264237F215843494200F0A9FF012336
:104000004000184310BD10B503211820FFF772FFC0
:104010007F2801DD0138FF3803007F3301DA7F207C
:10402000404264237F215843494200F091FF01231D
:104030004000184310BD002070470020704700204A
:104040007047002070470020704700207047002014
:1040500070470020704770477047704710B5034A9B
:1040600008210348FEF7F8FB10BDC04608010020F8
:104070001771000010B5FFF739FAAF20C000FDF747
:10408000ABFFFEF75BFC0448FEF7ACFDFEF7B2FAAF
:10409000FEF714FE10BDC046D56C000010B5FDF74C
:1040A0002DFF10BD70B5002504AC24780573A9421E
:1040B00005D10A4B0A4A23210A4801F061F8016040
:1040C0000949920052589B0002715B588371A3000A
:1040D0005B58856043710223C37170BD9A71000003
:1040E0005D710000A871000030720000037B002B9E
:1040F00004D143738373036101330373704700007A
:104100001FB50191A02100240068C900D2B244501B
:10411000012A07D0A24203D0032A05D1042202E0DB
:10412000022200E006221343034A8350034B019A04
:10413000C250012343501FBD540500002405000058
:1041400010B50400FFF7D2FFA1222368A179D200A5
:1041500099506179064A200099502179043299508A
:10416000044B19685A689B68FFF7CAFF10BDC04628
:104170000C050000F40F00204BB2002B0CDB802359
:104180003F290CD81F290CD80F290CD807290CD887
:1041900003290CD81B060BE080239B0408E0DB04FA
:1041A00006E01B0504E05B0502E09B0500E0DB0583
:1041B0000168014A8B507047240500000368074AD4
:1041C00099501A00FC32D1680029FCD0A321C90003
:1041D00058580023C0B2D3607047C0461C05000089
:1041E00007B58022074BD2051A6000229A6002327E
:1041F0001A7111230E320093034905330348FFF768
:1042000051FF07BDF40F00200030004000100020D7
:10421000F8B505000E0017000024BC4208D02B683A
:10422000315D1B6828009847002801D00134F4E76D
:104230002000F8BD704710B51C3000F0D5FB10BD54
:1042400010B51C3000F0C2FB10BD70B5437E0D00F0
:10425000002B05D06430040000F0D5FB002801D00D
:10426000002004E02000290000F0A1FB012070BD27
:1042700010B51C3000F0BEFB10BD0000F7B5019377
:10428000FA23002504009B0083600D4B4560083332
:1042900003601C300F00160000F07EFB200064302D
:1042A00000F07AFB074AB600B35827616375019B9B
:1042B00020009B009B586576A576A375FEBDC04681
:1042C00010720000307200000123A022C375837DAC
:1042D0000C49C133FF33D2059B009950437DC13354
:1042E000FF339B009950CC210369074A4904995038
:1042F0000521243A9950817D08329950417D034A25
:10430000995070470C060000240500000C050000C1
:10431000F7B5050000200C00019382425CD0161E08
:10432000402E00D940262F001C37380000F04AFBF1
:10433000B1222B69D20080219C50012289005A5061
:10434000A97E002901D11A621A600024731E2A690D
:10435000A34206D1019B002B03D0802302219B00A6
:10436000D150012313621300FC33D968002902D114
:10437000996A0029F9D0996A00290AD1D960A32342
:10438000DB00D1583800C9B2013400F010FBA6425E
:10439000DCD8019A2B69002A04D11A00FC32916AF8
:1043A00000290AD001210022AA7659611900FC31A6
:1043B00088680028FCD08A6007E00121A976D961CD
:1043C000D16C0029FCD00021D164FC339A6A002A08
:1043D00001D000229A62E0B2FEBD10B50123FFF7C2
:1043E00097FF10BD0300AC3310B5040019706430A2
:1043F00000F0E8FA0123637610BD0000F8B5002252
:104400000D0001004276AC31036904000878B12147
:10441000C9005850802189005A5001321A629A60AE
:1044200026006436300000F0DFFA00280ED030009D
:10443000276900F0CBFA1E4BF8502369FC331A6A47
:10444000002A0CD19A6A002AF9D008E02369002DCD
:104450000AD11A00FC32916A002905D10EE09A6A4D
:10446000002AF3D11A62DBE701225A611A00FC32FA
:1044700091680029FCD00021916006E00121D961FA
:10448000D16C0029FCD00021D1641A000020FC323C
:10449000916A81420BD0074990625A5802305A50B3
:1044A000824204D0043A534253410230C01AF8BD4C
:1044B0001C050000C404000010B50121FFF79EFF99
:1044C00010BD000010B51323122202490248FFF765
:1044D000D5FE10BD004000401410002003210A4802
:1044E00002680A430260094802680A4302600849F8
:1044F000084A094B9B1A03DD043BC858D050FBDC2B
:1045000000F0B4F9FBF736FE2405004054050040E6
:10451000C07400000000002014020020FEE7FEE747
:10452000FEE7FEE7FEE7FEE7014B18607047C04676
:1045300050010020F7B500231E2877D83C4B80009F
:10454000C258042A14D006D8022A0DD00ED804234B
:10455000012A14D069E0062A0ED00BD31A2A0DD0F6
:1045600002231B2A0BD060E0082308E0102306E09A
:10457000202304E0402302E0802300E001232D4AB1
:104580001268082A04D9092A05D00A21022404E065
:104590000821002401E011000124A02501261C2788
:1045A0002548ED004651254D254E2D681B02AD00D6
:1045B0003D400195234D2D6800958559AC466746D1
:1045C000214D3D401D4385518359C0259C46009B8C
:1045D000AD021D40FF2367461B023B402B43019D5C
:1045E0001D43009B5F0160231F402B003B431C4386
:1045F00001238451154C036063680F48002BFBD0E6
:104600000024124B01255C60A123DB00C3584560E8
:10461000A025ED0044511BB2914207D002D98A1A5D
:10462000D34003E0521A934000E000231800FEBD7F
:104630003072000054010020007000404C01002046
:104640000405000048010020FF00FFFFFC7000404F
:10465000F0B51E286CD8374B8000C258364B1E6808
:10466000002E2ED1C2243548A4000759344B03250F
:104670003B40C0273F023B4303518023893C9B00C2
:10468000FF3C03512F4F03602F4B803CD859FF3C18
:10469000A043D8510437D859A8432043D8510837EC
:1046A000D8590C35A843083D2843D851A820C0004C
:1046B0001E508026C120760280001E501C601E4BBA
:1046C0001C6000231426214834005C432558040054
:1046D0006F1C0FD1142058432250A0200325C13253
:1046E000FF329200C0051550194A08001268082AC6
:1046F00003D10BE0AA4218D1ECE7082A02D9083A04
:10470000D14002E00820821A91400800142253434D
:10471000E3189A680C495132FF32920058605050A9
:10472000DA68C1239B00CA5002E00133032BCBD1CE
:10473000F0BDC04630720000CC10002000E100E067
:10474000FF00FFFF0405000000900040580100201A
:10475000500100201E4BF0B5596C18001D4A00296D
:1047600014D0A025A12600230124ED05F600D15880
:104770004F1C06D0D7187F68002F02D027008F402B
:10478000AF5114333C2BF2D100234364131DA025F9
:1047900040329446002001240F4EED05DA680F499F
:1047A000920057180A495218526C002A0CD01A1F4E
:1047B0001268511C05D01968FF2902D021009140D0
:1047C000A9513A00FC32506414339C45E6D1F0BD47
:1047D000FC900040580100200C05000000900040B3
:1047E00000B51E2816D80C4A83009B58032911D8FF
:1047F000A0220800C133FF33D2059B0000F014FB58
:1048000002080406002104E00C2102E0042100E07B
:104810000321D15000BDC046307200001E280DD8C3
:10482000074B8000C058A0220123D20583400029F5
:1048300001D1044901E0A121C90053507047C0468D
:10484000307200000C050000030000201E2B0AD867
:10485000A222A021D200C9058858034A9B009B5878
:10486000D840012318407047307200002D4B10B51E
:104870001A78012A19D12C4A1268120715D12B4A2D
:10488000E0241168F0220800104021420BD1284991
:104890000968114209D12749274A11608021274A16
:1048A0000902116001E03028F1D01A78012A0DD1F7
:1048B0001D490968090709D1F0201C490968014010
:1048C000402903D11A490968014223D01B68DBB291
:1048D000012B25D1144B1B681B0721D1134B1A68E0
:1048E000F0231A40A02A04D1114A12681A4203D0B8
:1048F00016E0D02A14D1F7E7114B1A68012A03D128
:10490000C022104B1A600BE00F4A1A601A68012A85
:10491000FCD1F5E7C1218020C900C0054250D5E790
:1049200010BDC046E00F00F0E40F00F0E80F00F00B
:10493000EC0F00F0DFFF07C004050040186C0040DA
:1049400000EC064014EC064075930000F7B5060035
:104950000D000C008B180193019B671B9C4207D034
:10496000336821781B683000984701340028F3D160
:104970003800FEBD70B505000C00081E07D001F020
:10498000B5F82B6802005B6821002800984770BDCD
:1049900010B5FFF7EFFF10BD10B540220021040055
:1049A00000F077FC002320002364636410BD3F23E4
:1049B000026C10B5541C2340446C9C4201D08154BD
:1049C000036410BD0023036443647047436C026CAE
:1049D000934206D03F21C25C01330B404364100078
:1049E00001E0012040427047036C406C181A00D56A
:1049F00040307047436C026C934201D0C05C01E0D0
:104A0000012040427047036C406C5A1C3F23134006
:104A1000181A42424241D0B270470120704710B587
:104A200003681322DB69984710BD70470369054A84
:104A30009950FC331A6A002AFCD0002201201A6225
:104A40007047C0461C050000030010B55C331A789F
:104A50001F2313400122110099400D4B0424D967F4
:104A6000C221036989005C505A60DA60A0220021EB
:104A7000D20099500122074952425A500649143037
:104A80005A500C395A5008315A50FFF79BFF10BD4D
:104A900004E100E00C0500001405000010B514301E
:104AA000FFF7A2FF10BD10B51430FFF7A3FF10BD34
:104AB00010B51430FFF78AFF10BD0000030070B579
:104AC0005E331C780269604BD45003005D331C7860
:104AD0005E4BD450030061331C785D4B012C0CD12C
:104AE00005005F352E78A225ED0056510500603592
:104AF0002E78A125ED00565100E00024D4509623D5
:104B0000DB00994238D996231B01994237D9962365
:104B10005B01994236D996239B01994234D9E1230E
:104B20009B01994232D99623DB01994231D9E12385
:104B3000DB0199422FD996231B0299422DD9E123FB
:104B40001B0299422BD996235B02994229D9E12372
:104B50005B02994227D9E1239B02994225D93D4B1B
:104B6000994224D9E123DB02994223D9E1231B0393
:104B7000994221D8384B21E09E23DB021EE09D2381
:104B80001B031BE0354B19E0354B17E0EC239B036F
:104B900014E0344B12E0344B10E0344B0EE0344B55
:104BA0000CE0344B0AE0344B08E0344B06E0802341
:104BB000DB0403E0324B01E080235B053149002434
:104BC00053500423243953501100FC31CC600C6243
:104BD000C1210134890014605C3094605350037823
:104BE0001F202200D9B20840824080342648FF347A
:104BF0005BB20251002B13DA0F230B40083B234C0E
:104C00009B089B001B1903242140A140FC348C40CD
:104C1000DD69A543C0248C4021002943D96111E0FE
:104C2000194C9B089B001B1903242140A140C0255F
:104C3000FC348C40AD005E59A643C0248C4021005A
:104C400031435951026070BD0C050000140500008D
:104C50006C05000090D0030000D0BE0E00B0130021
:104C60000050270000A04E0000F0750000509D008D
:104C700000F0EB0000903A0100E0D70100B0AF0374
:104C800000705F072405000000E100E000ED00E097
:104C9000F7B5009308AB1B7800250193FA230400B5
:104CA0009B0083600E4B45600833036014300F0097
:104CB0001600FFF771FE23005C3327611E70009B16
:104CC000084A9B00995823005D331970019B20000E
:104CD0009B009A5823005E33DD701A70FEBDC046FB
:104CE000AC72000030720000036910B51A00FC328B
:104CF000D2680400002A0AD0A322D20099581430A6
:104D0000C9B2FFF754FE00222369FC33DA6010BDFC
:104D100010B50248FFF7E8FF10BDC046D0100020D4
:104D20001D2307B502220093024901330248FFF711
:104D3000AFFF07BD00200040D010002070470000EA
:104D400010B500F047F8FFF7F9FF012000F024F854
:104D5000FFF790F9FFF7A2F9024B002BFAD000E021
:104D600000BFF7E700000000084A0949094B10B5E9
:104D70001B688858FA22190A1B0618439200002360
:104D800000F0D2F94904C00B084310BD040500002F
:104D9000001001403411002070B5041E09D0FFF747
:104DA000E3FF050000F014F8FFF7DEFF401B84422C
:104DB000F8D870BD0022044B9A60044A136801338E
:104DC000DBB213607047C046FC1001403411002074
:104DD00070470000C421114A89005058104B03400D
:104DE000C020000203435350802391399B02FF39B6
:104DF000535013608023A3220021DB05D200995079
:104E00000122A1209A60074BC0001950C120023135
:104E100080001950403019501A60704700E100E0DE
:104E2000FF00FFFF0010014002B47146490849002D
:104E3000095C49008E4402BC7047C046002243080A
:104E40008B4274D303098B425FD3030A8B4244D352
:104E5000030B8B4228D3030C8B420DD3FF22090294
:104E600012BA030C8B4202D31212090265D0030B53
:104E70008B4219D300E0090AC30B8B4201D3CB0349
:104E8000C01A5241830B8B4201D38B03C01A52418B
:104E9000430B8B4201D34B03C01A5241030B8B428D
:104EA00001D30B03C01A5241C30A8B4201D3CB0278
:104EB000C01A5241830A8B4201D38B02C01A52415D
:104EC000430A8B4201D34B02C01A5241030A8B4260
:104ED00001D30B02C01A5241CDD2C3098B4201D378
:104EE000CB01C01A524183098B4201D38B01C01AF6
:104EF000524143098B4201D34B01C01A524103096D
:104F00008B4201D30B01C01A5241C3088B4201D31B
:104F1000CB00C01A524183088B4201D38B00C01AC8
:104F2000524143088B4201D34B00C01A5241411AEF
:104F300000D20146524110467047FFE701B50020FC
:104F400000F0F0F802BDC0460029F7D076E77047C0
:104F500003460B437FD4002243088B4274D30309DA
:104F60008B425FD3030A8B4244D3030B8B4228D37B
:104F7000030C8B420DD3FF22090212BA030C8B42A1
:104F800002D31212090265D0030B8B4219D300E041
:104F9000090AC30B8B4201D3CB03C01A5241830BC6
:104FA0008B4201D38B03C01A5241430B8B4201D376
:104FB0004B03C01A5241030B8B4201D30B03C01A9F
:104FC0005241C30A8B4201D3CB02C01A5241830A19
:104FD0008B4201D38B02C01A5241430A8B4201D348
:104FE0004B02C01A5241030A8B4201D30B02C01A72
:104FF0005241CDD2C3098B4201D3CB01C01A5241D9
:1050000083098B4201D38B01C01A524143098B4261
:1050100001D34B01C01A524103098B4201D30B014A
:10502000C01A5241C3088B4201D3CB00C01A52416F
:1050300083088B4201D38B00C01A524143088B4234
:1050400001D34B00C01A5241411A00D201465241CD
:10505000104670475DE0CA0F00D04942031000D3EC
:105060004042534000229C4603098B422DD3030A41
:105070008B4212D3FC22890112BA030A8B420CD351
:10508000890192118B4208D3890192118B4204D37A
:1050900089013AD0921100E08909C3098B4201D3FA
:1050A000CB01C01A524183098B4201D38B01C01A34
:1050B000524143098B4201D34B01C01A52410309AB
:1050C0008B4201D30B01C01A5241C3088B4201D35A
:1050D000CB00C01A524183088B4201D38B00C01A07
:1050E0005241D9D243088B4201D34B00C01A5241DE
:1050F000411A00D20146634652415B10104601D36B
:105100004042002B00D54942704763465B1000D3F4
:10511000404201B5002000F005F802BD0029F8D09A
:1051200016E770477047C046F0B54F464646C0B4D4
:105130001604360C9946330005042C0C070C150C8C
:1051400063437E436F4365431C0CAD1964199C4651
:10515000A64203D980235B02984647446346250C48
:10516000EF191D044B464A4343432D0C2404641994
:105170009918C91920000CBC90469946F0BDC0464C
:105180007FB51D000A4B06001B68D868002A02D1B3
:10519000084C230001E01300074C029300913300F8
:1051A0002A000649019400F021F800F023FEC046D1
:1051B000F40100206C6B0000DC720000E97200005A
:1051C000084B10B50400002B02D0002100E000BF06
:1051D000054B1868836A002B00D09847200001F027
:1051E000F3FAC046000000001C7300000EB403B5C3
:1051F000010003AB044804CB0068019300F016F9EA
:1052000002B008BC03B01847F40100200E4B70B583
:1052100000251E000D4CE41AA410A54204D0AB00DA
:10522000F35898470135F8E701F0D0FA084B00250C
:105230001E00084CE41AA410A54204D0AB00F35899
:1052400098470135F8E770BDFC010020FC01002003
:10525000FC0100200C02002010B5034B010018686F
:1052600000F066F810BDC046F401002010B5034BF5
:105270000100186800F016F810BDC046F4010020C7
:10528000002310B59A4203D0CC5CC4540133F9E733
:1052900010BD03008218934202D019700133FAE75F
:1052A0007047000030B500293ED004390B68002B50
:1052B00000DAC9181D4A13681400002B02D14B6094
:1052C000116031E08B420DD90A688818834203D1FE
:1052D00018685B6882180A604B60216024E08A428B
:1052E00003D813005A68002AF9D11D685C198C4252
:1052F0000BD10968691858181960824214D11068D6
:105300005268411819605A600EE08C4202D90C2391
:10531000036009E008680C18A24203D114685268BF
:10532000201808604A60596030BDC0463C1100201A
:10533000032370B5CD1C9D43083506000C2D01D20A
:105340000C2505E0002D03DA0C230020336040E03B
:10535000A942F9D81F4B1C681A002100002913D05C
:105360000B685B1B0DD40B2B02D90B60CC181EE015
:105370008C4202D1636813601AE04B6863600C00D2
:1053800016E00C004968E9E7134C2368002B03D1B1
:10539000300000F033FB20602900300000F02EFBCD
:1053A000431CD1D00323C41C9C43A0420AD12560D6
:1053B000200007220B30231D9043C31A09D05A4204
:1053C000E25006E0211A300000F018FB431CEED139
:1053D000BAE770BD3C11002038110020936810B569
:1053E000013B9360002B05DA9469A34208DBCBB242
:1053F0000A2B05D01368581C10601970C8B201E060
:1054000000F02CFC10BDF8B506000F001400D518F4
:10541000AC4208D021783A003000FFF7DFFF0134BA
:10542000431CF5D100E00020F8BD0000F0B59FB0AE
:1054300006000F0002920593002804D08369002B18
:1054400001D100F0D3FD7F4B9F4201D1776808E086
:105450007D4B9F4201D1B76803E07C4B9F4200D156
:10546000F768BB891B070AD53B69002B07D00023CF
:1054700006AD6B6120336B761033AB763DE03900BF
:10548000300000F043FC0028F1D001204042D6E07B
:10549000059A111D12680591002A00DA7FE0099231
:1054A000013423782E2B00D18DE021780322684827
:1054B00000F082FE002807D0654B2A68C01A4023FE
:1054C000834013432B6001342178631C062261481A
:1054D0000293297600F070FE002800D19DE05E4B1B
:1054E000002B00D090E00722059B0733934308333D
:1054F00005936B69039A9B186B61029C2378002BC0
:1055000004D1029BE31A049312D003E0252BF8D0B8
:105510000134F3E7049B029A39003000FFF773FF70
:10552000431C00D186E06A69049B944663446B6126
:105530002378002B7ED00122002352426A6002A908
:105540005432521801342B60EB60AB601370AB65C2
:1055500021780522414800F02FFE002808D03F4B5B
:105560002A68C01A0123834013432B600134EFE7FC
:105570002B68DA0604D55322202102A812181170D4
:105580001A0704D553222B2102A812181170227871
:105590002A2A00D17CE7099B00200A2105E052421B
:1055A000EA60022213432B607AE72278303A092A14
:1055B00004D84B4301349B180120F6E7002800D1A2
:1055C0006FE709936DE763782A2B0AD1059B0234B4
:1055D0001A1D1B680592002B01DA01235B42079319
:1055E00063E700230A201A0001346B602178303908
:1055F000092904D84243013452180123F6E7002B4D
:1056000000D152E7079250E705AB00933A00144BE4
:105610002900300000E000BF07E005AB00933A002E
:105620000F4B2900300000F08BF80390039B0133EF
:1056300000D05EE7BB895B0600D526E70B981FB05C
:10564000F0BDC046547400007474000094740000EF
:10565000267300002A730000000000002073000081
:1056600007540000F7B5170001938A680B69009092
:105670000C00934200DA130022003B6043321278A0
:10568000002A01D001333B6023689B0602D53B68AA
:1056900002333B60062523681D401ED023004333A0
:1056A0001B785A1E9341226892061CD53020E118BF
:1056B0004331087021005A1C45310978A218433241
:1056C000023311700FE02200012319320199009872
:1056D000089EB047431C0ED00135E3683A689B1A18
:1056E0009D42F0DBDAE72200019943320098089DE1
:1056F000A847431C02D10120404220E00623206835
:10570000E1683A6803400025042B03D18D1AEB436E
:10571000DB171D40A3682269934201DD9B1AED1837
:105720000027BD420AD0220001231A3201990098B5
:10573000089EB047431CDED00137F2E70020FEBDD3
:10574000F0B58BB006920A0043320793059004929D
:105750000A7E0C00109B6E2A00D1ABE011D8632AA0
:1057600022D009D8002A00D1B5E0582A00D0C5E0DF
:1057700045310A70814A4FE0642A1DD0692A1BD046
:10578000BCE0732A00D1AAE009D86F2A29D0702A78
:1057900000D0B3E0202209680A43226037E0752A6E
:1057A0001FD0782A33D0A9E00E001A684236111DA6
:1057B000196013683370A4E021681A68080606D4DB
:1057C000490604D5111D19600023D55E02E0111DA4
:1057D00019601568002D3BDA2D23049A6D42137071
:1057E00036E021681A68080606D4490604D515680B
:1057F000111D1960ADB202E0111D196015685F4BF3
:10580000227E039308276F2A1DD00A271BE022005F
:105810007821453211705A4A19680392081D22688E
:1058200018600D68100602D4500600D5ADB2D3073B
:1058300002D520231A4322601027002D03D12023F4
:1058400022689A4322602300002243331A7002E048
:105850000A274A4B03936368A360002B09DB0422E9
:10586000216891432160002D05D1049E002B11D0A9
:105870007BE0002D79D0049E28003900FFF764FBFF
:10588000039B013E5B5C280033703900FFF7D6FABA
:10589000051EF1D1082F09D12368DB0706D56368FF
:1058A0002269934202DC3023013E3370049B9B1B30
:1058B00023612BE009681A68080607D4490605D554
:1058C000111D19601368A28A1A8004E0111D196065
:1058D000136862691A600023049E236116E01A6847
:1058E000111D1960166800216268300000F064FC28
:1058F000002801D0801B6060636803E02600423608
:105900003270012323610023049A1370079B09AAB4
:1059100000932100069B0598FFF7A4FE431C02D1CB
:105920000120404227E02369320006990598079D2F
:10593000A847431CF4D0236800259B070FD4099B7C
:10594000E068984217DA180015E0220001231932A6
:1059500006990598079EB047431CE1D00135E368DE
:10596000099A9B1A9D42F0DBE9E72600039B423629
:105970001B7833708EE70BB0F0BDC046317300006A
:1059800042730000154B10B51C68A36B002B15D19A
:105990001820FFF761FC124BA0630380114B01221A
:1059A0004380114B8380114BC380114B038105232E
:1059B000438106338381002302614361A46B0D4A56
:1059C000206961690C4BFFF7AFFB012200238018AF
:1059D0005941206161614800400810BDF401002078
:1059E0000E330000CDABFFFF341200006DE6FFFF69
:1059F000ECDEFFFF2D7F954C2DF45158002370B540
:105A0000064C05000800236000F0C8FE431C03D1CB
:105A10002368002B00D02B6070BDC04630240020CE
:105A20000CB430B5164B9DB00C1E1D6804DA8B23E8
:105A300001202B6040421DE0822302A99B008B8144
:105A40000023029008619C4200D0631E8B604B6172
:105A500001235B42CB81209A21AB2800019300F007
:105A600053FC431C01DA8B232B60002C02D0002353
:105A7000029A13701DB030BC08BC02B01847C04673
:105A8000F40100200EB410B59DB002A90290086187
:105A90000B48822488604861012040421FABC881C6
:105AA000084804CBA400006801938C8100F02CFC12
:105AB0000023029A13701DB010BC08BC03B0184735
:105AC000FFFFFF7FF401002002780B78002A03D04B
:105AD000013001319A42F7D0D01A7047031C0A787E
:105AE00001311A700133002AF9D170470023C25CDA
:105AF0000133002AFBD1581E7047030030B5002A3D
:105B00000DD00C7801335D1E013A2C700131002C50
:105B1000F5D19A189A4202D01C700133FAE730BDD1
:105B2000F0B51E00454B87B01B6801920293082216
:105B30000B00059003911C7802995D1C09194878A7
:105B4000104001D02B00F6E72D2C04D19D1C5C7871
:105B50000123009304E000902B2C01D15C789D1C64
:105B6000002E02D0102E0AD162E0302C5ED120220D
:105B70002B789343582B54D110266C780235009F14
:105B800031007B1E9F412E4BFF183800FFF7DCF9D8
:105B9000380004913100FFF751F900230322070078
:105BA00094461800029A121951780422114201D029
:105BB000303C07E06246114017D03722012900D05F
:105BC0002032A41AA64210DD5A1C0BD0B84207D8C6
:105BD00002D1049B9C4203DC70430123201801E0A6
:105BE00001235B422C780135DCE75A1C0BD100986D
:105BF000059A431E9841124BC01822231360019B43
:105C0000002B0AD117E0009A002A00D04042019AE6
:105C1000002A10D0039A002B00D06A1E019B1A6044
:105C200009E03024002EAAD10826A8E70A26A6E714
:105C3000302C9CD0A3E707B0F0BDC046F80100208F
:105C4000FFFFFF7F10B513000A0001000248006843
:105C5000FFF766FF10BDC046F4010020F8B505004F
:105C60000F001400002804D08369002B01D100F03C
:105C7000BDF9234B9C4201D16C6808E0214B9C424A
:105C800001D1AC6803E0204B9C4200D1EC68A369D1
:105C9000A360A3891B070AD52369002B07D02368BB
:105CA0002269FEB2981A636998420FDB08E021006E
:105CB000280000F02BF80028F1D0012040421DE020
:105CC0002100280000F024F90028F6D1A368013053
:105CD000013BA36023685A1C22601F7063699842CD
:105CE00005D0A3893000DB0708D50A2E06D1210094
:105CF000280000F00DF90028DFD13000F8BDC046C3
:105D0000547400007474000094740000354B70B536
:105D10001D6806000C00002D05D0AB69002B02D1D8
:105D2000280000F063F9304B9C4201D16C6808E018
:105D30002E4B9C4201D1AC6803E02D4B9C4200D11C
:105D4000EC68A3899AB2110723D4D10607D409229B
:105D50000120326037321343A381404240E05307B1
:105D600013D5616B002908D023004433994202D037
:105D70003000FFF797FA002363632422A38993433B
:105D8000A38100236360236923600822A38913434E
:105D9000A3812369002B0BD1A023A2899B00134070
:105DA00080229200934203D02100300000F0B2F92B
:105DB0000123A289134005D00023A36063695B42DD
:105DC000A36103E0910700D46369A3600020236905
:105DD000834205D1130603D540231A43A28101381B
:105DE00070BDC046F40100205474000074740000BB
:105DF0009474000010B5062000F0AEFB012000F006
:105E0000E3FC0000F7B58A8905000C0013075AD49B
:105E10004B68002B02DC0B6C002B19DDE76A002FAE
:105E200016D000232E682B6080235B011A4001D01E
:105E3000606D14E00123216A2800B847431C0ED18D
:105E40002B68002B0BD01D2B01D0162B02D12E60FE
:105E500000205AE04022A3891343A38155E0A3897F
:105E60005B0706D56368C01A636B002B01D0236CF7
:105E7000C01A00230200216A2800E76AB847A389F4
:105E8000421C06D129681D293AD8204ACA40D207A7
:105E900036D50022626022692260DB0405D5431CEE
:105EA00002D12B68002B00D16065616B2E60002948
:105EB000CED023004433994202D02800FFF7F2F9F4
:105EC0000020606321E00F69002FC1D00B680F60D4
:105ED000DB1B01930023920700D14B69A36003E011
:105EE000019B3F181B1A0193019B002BB0DD019B06
:105EF0003A00216A2800A66AB0470028F0DCA3898E
:105F0000402201201343A3814042FEBD01004020F6
:105F10000B6970B505000C00002B01D100201CE0BE
:105F2000002804D08369002B01D100F05FF80B4BEF
:105F30009C4201D16C6808E0094B9C4201D1AC68DD
:105F400003E0084B9C4200D1EC680C22A35E002BBE
:105F5000E4D021002800FFF755FF70BD5474000005
:105F6000747400009474000010B5024900F0B0F899
:105F700010BDC046115F0000002310B5040003608F
:105F80004360836081814366C281036143618361B1
:105F9000190008225C30FFF77CF9054B246263622C
:105FA000044BA362044BE362044B236310BDC04661
:105FB00099650000C1650000F965000025660000D4
:105FC00070B568254B1E5D430E0029007431FFF744
:105FD000AFF9041E08D000212A00016046600C3091
:105FE000A0606832FFF755F9200070BD836913B5D2
:105FF0000400002B28D18364C3640365134B144A47
:106000001B6882620193984201D1012383612000C1
:1060100000F020F86060200000F01CF8A060200074
:1060200000F018F80022E06004216068FFF7A4FF88
:1060300001220921A068FFF79FFF02221221E068D8
:10604000FFF79AFF0123A36113BDC0461C73000034
:10605000695F0000F8B51D4B06001D68AB69002B99
:1060600002D12800FFF7C2FF4835AC686B68013BDE
:1060700005D40C22A75E002F10D06834F7E72B68F8
:10608000002B01D02D68F0E704213000FFF798FFC6
:1060900028600028F6D10C23336016E0012320008D
:1060A0005B42E3810233A38167662760A760676074
:1060B00027616761A7615C3008223900FFF7E9F8C2
:1060C00020006763A763A764E764F8BD1C73000042
:1060D000F7B504000700002601914834002C16D0C3
:1060E0006368A5680093009B013B00930DD4AB89C6
:1060F000012B08D90E22AB5E013304D029003800F1
:10610000019B984706436835EDE72468E6E73000D1
:10611000FEBD0000F0B58B8991B006000C009B0716
:1061200026D40E23C95E002904DA8023A5891D40E8
:1061300010D10CE001AA00F0A1FA0028F5DBF02351
:10614000029D1B021D401A4BED186B425D418027DA
:10615000FF0001E00025402739003000FFF7E8F894
:1061600000280CD1A3899A051FD402221343A381CE
:1061700023004733236023610123636115E08022FC
:106180000C4BB362A38920601343A3812061676134
:10619000002D0AD00E23E15E300000F081FA0028C5
:1061A00003D00122A3891343A38111B0F0BDC046DF
:1061B00000E0FFFF695F0000C9B28218904204D07E
:1061C00003788B4202D00130F8E70020704710B509
:1061D000884202D98B18984201D3002305E09B1A0C
:1061E000013A08D3995C8154FAE7934203D0CC5C1E
:1061F000C4540133F9E710BDF8B506000C001500D2
:10620000002904D11100FFF793F8040018E0002AD8
:1062100003D1FFF747F82C0012E000F067FA85423F
:106220000ED929003000FFF783F8071E07D02100A0
:106230002A00FFF725F821003000FFF733F83C0073
:106240002000F8BDF0B58E6885B007000C00039201
:1062500001939E4243D890238A89DB001A423ED0A4
:1062600003250969236801985B1A029363695D43FA
:10627000EB0F5D19029B6D1001331B18AB4200D967
:106280001D00530510D529003800FFF751F8061EF0
:1062900014D0029A2169FEF7F3FFA289194B13402B
:1062A00080221343A38112E02A003800FFF7A4FFE5
:1062B000061E0CD121693800FEF7F4FF0C234022A2
:1062C00001203B60A38940421343A38117E0029B56
:1062D0002661F61826606561019EED1AA560019B96
:1062E000B34200D21E00320003992068FFF76FFF0F
:1062F0000020A3689B1BA36023689E19266005B03D
:10630000F0BDC0467FFBFFFFF0B59FB00290059344
:106310008B890F0016001B0610D50B69002B0DD1C1
:106320004021FFF705F838603861002804D10C23BC
:10633000029A01381360D8E040237B61002306AD48
:106340006B6120336B761033AB7634002378002BEF
:1063500003D1A31B049312D003E0252BF9D0013401
:10636000F4E7A31B320039000298FFF76BFF431CD0
:1063700000D1B4E06A69049B944663446B6123785E
:10638000002B00D1ABE00122002352426A6002A937
:106390005432521801342B60EB60AB601370AB6564
:1063A000534E217805223000FFF706FF002807D062
:1063B0000123801B83402A68013413432B60EFE7DD
:1063C0002B68DA0604D55322202102A81218117076
:1063D0001A0704D553222B2102A812181170227813
:1063E0002A2A03D0099B00200A210EE0059A111DDC
:1063F00012680591002A01DB099204E05242EA602A
:10640000022213432B6001340BE02278303A092A30
:1064100004D84B4301349B180120F6E7002800D034
:10642000099323782E2B1ED163782A2B0AD1059B42
:1064300002341A1D1B680592002B01DA01235B420E
:10644000079310E000230A201A0001346B602178C2
:106450003039092904D84243013452180123F6E7A0
:10646000002B00D00792234E217803223000FFF743
:10647000A3FE002806D04023801B83402A680134F5
:1064800013432B60217806221B48661C2976FFF7F0
:1064900093FE002812D0194B002B06D10722059B32
:1064A000073393430833059314E005AB00933A0098
:1064B000134B2900029800E000BF07E005AB0093F2
:1064C0003A000F4B29000298FFF73AF90390039B1B
:1064D000013304D06B69039A9B186B6135E7BB8964
:1064E0000B985B0601D5012040421FB0F0BDC046AD
:1064F00020730000267300002A73000000000000D3
:106500004562000070B504000D1E1F2D04D916232E
:106510000360012040421EE0426C002A04D08B0040
:10652000D2181368002B08D1200000F031F82A009F
:106530000100200000F01AF80DE00020012B0AD025
:10654000591C03D117332360013004E000242800D4
:1065500014609847200070BD10B5034B0100186807
:10656000FFF7D0FF10BDC046F4010020002370B536
:10657000064C050008001100236000F0F7F8431CEA
:1065800003D12368002B00D02B6070BD3024002085
:1065900010B500F0DBF810BD70B50C000E25495F9A
:1065A00000F0B0F8002803DB636D1B18636503E09F
:1065B000A289024B1340A38170BDC046FFEFFFFFCD
:1065C000F8B51F008B8905000C001600DB0505D50A
:1065D0000E23C95E0022022300F074F8A289054B45
:1065E00028001340A38132000E23E15E3B0000F03F
:1065F0001FF8F8BDFFEFFFFF70B50C000E25495FD7
:1066000000F060F8A389421C03D1054A1340A3811E
:1066100004E0802252011343A381606570BDC0462F
:10662000FFEFFFFF10B50E23C95E00F015F810BD97
:1066300070B50500080011000022064C22601A0007
:1066400000F0BAF8431C03D12368002B00D02B6064
:1066500070BDC04630240020002370B5064C0500F4
:106660000800236000F062F8431C03D12368002B6C
:1066700000D02B6070BDC04630240020002370B5D0
:10668000064C050008001100236000F057F8431C79
:1066900003D12368002B00D02B6070BD3024002074
:1066A000002370B5064C05000800236000F056F882
:1066B000431C03D12368002B00D02B6070BDC04663
:1066C0003024002070B50500080011000022064C9F
:1066D00022601A0000F052F8431C03D12368002BFB
:1066E00000D02B6070BDC046302400200B1F1A68FC
:1066F000101F002A04DA891804390B68D0180438EE
:106700007047000070B50500080011000022064C1B
:1067100022601A0000F03AF8431C03D12368002BD2
:1067200000D02B6070BDC0463024002058220120CC
:10673000014B40421A60704730240020582201204B
:10674000014B40421A60704730240020582201203B
:10675000014B40421A607047302400205822024BFF
:1067600000201A607047C0463024002058220120C3
:10677000014B40421A60704730240020582201200B
:10678000014B40421A6070473024002058220120FB
:10679000014B40421A60704730240020044A1368BD
:1067A000002B03D01818106018007047014BF9E750
:1067B000401100203824002058220120014B404283
:1067C0001A60704730240020FEE7C046F8B5C04686
:1067D000F8BC08BC9E467047F8B5C046F8BC08BC7B
:1067E0009E467047F6060000880600000607000077
:1067F0003C07000078070000B2070000EE07000029
:1068000016080000540800009A080000F60800006E
:106810003A090000A0090000EC090000140A000079
:106820004E0A0000980A0000C00A0000F80A0000A2
:10683000300B00006C0B0000F20B0000BA0C0000E3
:10684000480D0000A60D0000E80D00000A0E000033
:10685000120E0000F40E0000F6060000F60600001E
:10686000F6060000F6060000400F0000AA0F000028
:10687000141000005E100000C0100000461100005F
:10688000CE1100001C12000066120000AC120000C5
:10689000F81200004413000090130000DE13000003
:1068A0003414000072140000DE1400000E15000005
:1068B0005A150000A6150000F21500002C16000065
:1068C00078160000F6060000F6060000F606000046
:1068D000F6060000C4160000F4160000241700009D
:1068E0005017000080170000AC170000F6060000EB
:1068F000F6060000F6060000F6060000E4170000A9
:106900002C18000078180000A8180000D418000007
:10691000021900004C190000F6060000F6060000FF
:10692000F60600007A190000AA190000DA19000022
:106930000A1A0000361A0000661A0000921A0000B7
:10694000BC1A0000E61A0000161B0000461B0000DF
:10695000881B0000B41B0000E41B0000101C00009A
:10696000F6060000F6060000F6060000F606000037
:10697000F6060000401C00006C1C0000981C000083
:10698000C41C0000F01C0000281D0000601D000059
:10699000981D0000D01D0000FC1D00002A1E0000F4
:1069A0005A1E0000F6060000F6060000F60600007B
:1069B000F6060000F6060000F6060000F6060000E7
:1069C000F6060000F6060000F6060000F6060000D7
:1069D000F6060000F6060000F6060000881E00001D
:1069E000B61E000066616C73650074727565006C9C
:1069F000697374206F66202564206974656D730067
:106A00006F626A656374206F6620636C6173733AAA
:106A100020256400537461636B20756E6465726633
:106A20006C6F77000D0A564D2050616E69633A20F5
:106A300025730D0A00496E73756666696369656E34
:106A400074206D656D6F727920666F72204D696379
:106A5000726F426C6F636B73206F626A6563742040
:106A60006865617000496E73756666696369656E15
:106A700074206D656D6F727920666F72204D696349
:106A8000726F426C6F636B7320737461636B00622F
:106A90006164206F626A65637420617420256C6490
:106AA0000A0025783A20256420776F7264732C20C1
:106AB000636C61737349442025640A00486561640E
:106AC00065723A2025780A0009307825782C0A006A
:106AD00025642025642025642025640A0042616421
:106AE000207265636F726420666F756E64206475D2
:106AF00072696E6720696E697469616C697A617424
:106B0000696F6E210A004E6F7420656E6F7567683D
:106B100020726F6F6D206576656E20616674657298
:106B200020636F6D70616374696F6E0A00526573E4
:106B3000746F72696E672025642073637269707464
:106B4000732E2E2E0053746172746564002D2D2DEA
:106B50002D2D0A0050657273697374656E74204D33
:106B6000656D6F727920546573740A0A000A496E64
:106B7000697469616C697A696E67204D656D6F72C1
:106B8000790A004D656D6F727920696E7469746958
:106B9000616C697A65643B2077726974696E6720FD
:106BA0007265636F7264732E2E2E0A005265636FD6
:106BB0007264206174206F66667365742025643A80
:106BC0002025642025642025642025642028256450
:106BD00020776F726473290A0046696E616C3A20EF
:106BE00063757272656E7420256420757365642008
:106BF00025642063302025642063312025640A0049
:106C00006E6F6E6500726164696F006469736162C2
:106C10006C65526164696F006D657373616765527D
:106C200065636569766564007061636B6574526560
:106C30006365697665007061636B657453656E6446
:106C4000007265636569766564496E74656765722F
:106C50000072656365697665644D65737361676528
:106C60005479706500726563656976656453747202
:106C7000696E670073656E64496E7465676572005E
:106C800073656E64506169720073656E64537472EB
:106C9000696E67007365744368616E6E656C00733E
:106CA000657447726F757000736574506F776572A5
:106CB000007369676E616C537472656E6774680007
:106CC0004E6F2066726565207461736B20656E740B
:106CD000726965730057656C636F6D6520746F2012
:106CE0004D6963726F426C6F636B7321004D656D0C
:106CF0006F727920636C65617265642E00416C6C03
:106D0000207461736B732073746F707065640076A8
:106D10003035340020257320257300000700000063
:106D20000300000043616C6C696F706500686173FB
:106D3000546F6E6500706C6179546F6E65006861A8
:106D400073536572766F00736574536572766F0066
:106D50001500000001000000020000000400000017
:106D600005000000060000006E657400686173573E
:106D70006946690073746172745769466900737477
:106D80006F705769466900776966695374617475F5
:106D900073006D794950416464726573730074685F
:106DA000696E674465736372697074696F6E0063BE
:106DB0006C6561725468696E67446573637269706B
:106DC00074696F6E00617070656E64546F546869A9
:106DD0006E674465736372697074696F6E000D0E3F
:106DE0000F04050C0B0A060708090D0E0F04050C0D
:106DF0000B0A06070809646973706C6179006C6995
:106E00006768744C6576656C000000000000000047
:106E10000100000002000000030000000400000068
:106E20000500000006000000070000000800000048
:106E3000090000000A0000000B0000000C00000028
:106E40000D0000000E0000000F0000001000000008
:106E500012000000140000001600000018000000DE
:106E60001A0000001C0000001E00000020000000AE
:106E70002300000026000000290000002C00000074
:106E80002F00000032000000360000003A00000031
:106E90003E00000042000000460000004B000000E1
:106EA00050000000550000005A0000006100000082
:106EB000680000006F000000760000007D00000008
:106EC000840000008B000000920000009900000088
:106ED000A0000000A7000000AE000000B500000008
:106EE000BC000000C3000000CA000000D100000088
:106EF000D8000000DF000000E6000000ED00000008
:106F0000F4000000FB000000FF0000000000000093
:106F10000008080800080A4A4000000A5FEA5FEA21
:106F20000ED92ED36E19324489330C924C924D08EF
:106F30000800000004880808040804848488000A03
:106F4000448A4000048EC480000000048800000EC3
:106F5000C000000000080001224488100C92525228
:106F60004C048C84848E1C824C901E1EC244924C15
:106F700006CA525FE21FF01EC13E02448ED12E1F90
:106F8000E24488100ED12ED12E0ED12EC4880008D6
:106F900000080000048004880244880482000EC0B7
:106FA0000EC008048244880ED126C0040ED135B329
:106FB0006C0C925ED2521C925C925C0ED010100E41
:106FC0001C9252525C1ED01C901E1ED01C90100EA3
:106FD000D013712E12525ED2521C8808081C1FE278
:106FE00042524C1254981492101010101E113B75FE
:106FF000B131113935B3710C9252524C1C925C90E4
:10700000100C92524C861C925C92510ED00C825CF9
:107010001FE4848484125252524C1131312A44119B
:107020003135BB7112524C9252112A4484841EC4D1
:1070300088101E0EC808080E10080482410EC242B5
:10704000424E048A400000000000001F0804800037
:1070500000000ED2524F10101C925C000ED0100E89
:1070600002424ED24E0C925C900E06C81C88080E4E
:10707000D24EC24C10101C92520800080808024060
:1070800002424C10149814920808080806001B7558
:10709000B131001C925252000C92524C001C925C76
:1070A00090000ED24EC2000ED010100006C80498F8
:1070B00008080EC807001252524F0011312A44002E
:1070C000113135BB00124C8C9200112A4498001EDD
:1070D000C4881E06C48C8486080808080818080C92
:1070E000881800000C836073656E736F7273007490
:1070F000656D70657261747572650074696C745841
:107100000074696C74590074696C745A00746F75FA
:107110006368526561640074667400656E61626CD8
:1071200065446973706C6179007365745069786542
:107130006C006C696E65007265637400726F756EC9
:107140006465645265637400636972636C6500749E
:107150007269616E676C650074657874005350499C
:10716000436C6173733A3A535049436C61737328AB
:107170004E52465F5350495F547970652A2C2075F2
:10718000696E74385F742C2075696E74385F742C66
:107190002075696E74385F742900705F73706920A0
:1071A000213D204E554C4C002F55736572732F6A4C
:1071B0006F686E6D616C6F6E65792F4C696272617C
:1071C00072792F41726475696E6F31352F7061630A
:1071D0006B616765732F73616E646565706D69734C
:1071E0007472792F68617264776172652F6E52468E
:1071F000352F302E362E302F6C69627261726965C0
:10720000732F5350492F5350492E63707000000064
:1072100000000000000000004B420000114200008E
:107220003742000041420000714200003542000038
:107230000000000001000000020000001600000035
:107240000400000005000000060000000700000028
:1072500008000000090000000A0000000B00000008
:107260000C0000000D0000000E0000000F000000E8
:107270001A0000001B0000001400000013000000B2
:107280001100000003000000100000001C000000BE
:107290001D0000001E00000012000000150000008C
:1072A0001700000018000000190000000000000096
:1072B000000000002D4A00004D4900009D4A0000DA
:1072C000B14A0000A74A00002B4A00001F4A0000F4
:1072D000BD4A0000494A00001B4A00002C20667588
:1072E0006E6374696F6E3A200061737365727469BE
:1072F0006F6E2022257322206661696C65643A20D6
:1073000066696C6520222573222C206C696E6520CD
:107310002564257325730A004300000094010020B2
:10732000232D302B2000686C4C006566674546476E
:1073300000303132333435363738394142434445F1
:107340004600303132333435363738396162636460
:1073500065660000202020202020202020282828CA
:10736000282820202020202020202020202020200D
:107370002020202088101010101010101010101055
:107380001010101004040404040404040404101075
:107390001010101010414141414141010101010112
:1073A00001010101010101010101010101010110BE
:1073B00010101010104242424242420202020202E7
:1073C000020202020202020202020202020202108F
:1073D000101010200000000000000000000000005D
:1073E000000000000000000000000000000000009D
:1073F000000000000000000000000000000000008D
:10740000000000000000000000000000000000007C
:10741000000000000000000000000000000000006C
:10742000000000000000000000000000000000005C
:10743000000000000000000000000000000000004C
:10744000000000000000000000000000000000003C
:10745000000000000000000000000000000000002C
:10746000000000000000000000000000000000001C
:10747000000000000000000000000000000000000C
:1074800000000000000000000000000000000000FC
:1074900000000000000000000000000000000000EC
:1074A00000000000000000000000000000000000DC
:0874B0000000000000000000D4
:0874B800BC8CFF7F0100000005
:1074C000FFFFFFFF0B6C0000C5260000186C0000DA
:1074D000C9260000286C0000CD260000366C000094
:1074E000D1260000416C00008D260000516C000088
:1074F000A1260000656C000091260000746C00005D
:10750000D5260000806C0000D9260000896C0000A0
:10751000DD260000946C0000E12600009F6C000056
:10752000C1260000A86C000089260000B16C000094
:10753000992600002D6D0000AD320000356D000071
:10754000A93200003E6D0000B1320000476D00001E
:10755000B53200006C6D000065350000746D0000F0
:10756000893500007E6D000093350000876D0000B6
:107570009D350000926D0000A73500009E6D000053
:1075800073350000AF6D00007D350000C56D000053
:1075900069350000FE6D0000C935000018000000CC
:1075A000EF700000BD3F0000FB700000D73F0000FF
:1075B0000171000007400000077100008B3F0000D0
:1075C0000D710000E13D00001B7100003F40000014
:1075D0002971000043400000327100004740000064
:1075E000377100004B4000003C7100004F4000002C
:1075F00048710000534000004F7100003B40000004
:107600005871000037400000030000000200000035
:10761000080000000A000000FFFFFFFF000000005C
:10762000010000000000020001000000FFFFFFFF5A
:107630000000000002000000000004000200000042
:10764000FFFFFFFF00000000030000000000080033
:107650000300000000000000547400007474000077
:107660009474000000000000000000000000000012
:10767000000000001873000000000000000000007F
:1076800000000000000000000000000000000000FA
:1076900000000000000000000000000000000000EA
:1076A00000000000000000000000000000000000DA
:1076B0000000000094010020537300003901000015
:1076C000E1410000C5440000214D00000D01000013
:0476D00000000000B6
:04000003000044DDD8
:00000001FF
